:020000040800F2
:10500000F81B0020D55000089D8C0008E1820008A4
:105010000000000000000000000000000000000090
:10502000000000000000000000000000E99A0008F5
:10503000000000000000000065940008259C0008A6
:10504000E7500008E7500008E7500008E750000864
:10505000E7500008D95C0008E7500008E750000856
:1050600000000000E7500008015C0008E75000085D
:10507000E75000088D88000800000000E750000895
:1050800000000000E75000080000000000000000E1
:10509000E750000800000000E7500008E750000853
:1050A000E7500008E7500008E7500008A1A60008F4
:1050B000E7500008E7500008000000000000000072
:1050C0000348854600F0E8FC0048004715BA000890
:1050D000F81B00200448804704480047FEE7FEE72D
:1050E000FEE7FEE7FEE7FEE7C19C0008C1500008AE
:1050F00030B50B46014600202022012409E00D4670
:10510000D5409D4205D31D469540491B25469540F7
:1051100040191546521E002DF1DC30BDF0B51FB40C
:105120000646002082B005464024019100901BE015
:10513000019922460F46304600F098FB049A059BE1
:10514000801A994110D310461946224600F07EFB82
:10515000361A8F410197224601200021009F00F05E
:1051600075FB38184D4100902046641E0028DFDC96
:10517000019B00982946324607B0F0BD03460B4319
:105180009B0703D009E008C9121F08C0042AFAD2FD
:1051900003E00B780370401C491C521EF9D2704783
:1051A000D2B201E00270401C491EFBD270470022BF
:1051B000F6E710B513460A4604461946FFF7F0FF16
:1051C000204610BD30B504460020034600E05B1CBD
:1051D000934203D2E05CCD5C401BF8D030BDF8B503
:1051E00002464A40D40F42004B0052085B089A42E4
:1051F00002D20246084611464A0023D0C30D4A0097
:10520000DDB2120EAD1A202D35DA49020126490A07
:10521000F6058A19002C00D0524220214F1B11465E
:10522000B9402A411018C20D9A4221D0002C17D043
:10523000012D08DCDA05801AD20F8019D207DBB203
:1052400000F040FBF8BDDA05801A012340001B0680
:10525000C01880185A428018CA0F1043490007E04E
:105260004908C2071143DA05801A801940088018DE
:1052700000F020FBF8BD61000122511A001BF7E786
:105280000122D2075140AAE70122D2075040A6E7E7
:1052900070B502464A40D50F40004A00ED0740086D
:1052A0005208002814D0002A12D0C40DD30D410298
:1052B0000120C0055202490A520AE41A09181218BC
:1052C0007D34914201D3641C00E04900002C01DAD6
:1052D000002070BD0023914201D3891A0343400886
:1052E00049000028F7D100290AD0914202D10121BA
:1052F000C90705E0914201D2012101E00121C94322
:10530000E005C018401900F0D5FA70BD420005D084
:105310004200120E52428A4201DB00207047C9054A
:1053200008187047F0B507460846584087B0C00FC8
:10533000049048000E46590040084908BC1A8841AC
:1053400005D2384631461E4617460B4602465800DF
:10535000400810434CD0300D039040055900400DDB
:10536000490D0590401A0290402872DA1803012175
:10537000000B09050843019004980092002805D00D
:1053800001995242002088410092019002984021E8
:105390000A1A0199009800F059FA05460C466B4626
:1053A00007CB00F074FAC0197141039A0E0D002367
:1053B000D71756401A467A40164344D0049A002A1A
:1053C0002DD0029A012A039A15DC1205C01A9141C8
:1053D00001263605001C7141D20F059ED2070093AD
:1053E000019202962A46234600F0B2FA07B0F0BDB9
:1053F00038463146FAE71605224A0F46B218C01A57
:10540000B74101210905001C4F4100187F41114699
:1054100018187941E20F10436D19644113E0E20757
:105420006D0815436408C2071443039A0126120548
:10543000C01A91413605001C7141CE074008304327
:105440004908C01851412A46234600F074FACDE7B6
:10545000FFE7049801224000C117121A00238B4174
:1054600004983146C417381AA141EEE730B401243C
:10547000E407634030BC55E730B40124E4076140E1
:1054800030BC4FE70000E0FFF0B51FB488B00B99C7
:105490000998002448400999C00F4900490809911A
:1054A000C0070B990090490049080B910999089889
:1054B000A64608431CD00B990A98084318D00998AF
:1054C00001244000420D4800410D099824050003C5
:1054D000000B204309900B980003000B20430B9016
:1054E00050181C494018002201901446104605E04F
:1054F000002001460DB0F0BD032801DA034600E0AC
:1055000003239C46C11A0AAE0AE05F0008ADED5BBA
:105510004F00F75B7D430027AA187C41491C5B1EA6
:105520006145F2DD410004AB5A522104120C0A43DA
:10553000240C401C0828DFDB01980290009970467B
:1055400001910090059B049A0799069800F000FAD3
:10555000D0E700000DFCFFFFF0B50C465C4085B0C5
:10556000E40FE40703944C000026640859009446B5
:10557000490802460296224321D062460A431ED0C1
:105580006200570D4A000E032303550D0124024605
:105590002C492405781B1B0B360B4018234326434C
:1055A000614600901C46501AB44103D30098401C39
:1055B000009002E0921800985B41002803DA002076
:1055C000014605B0F0BD00200121090507468646C9
:1055D00011E064461D46141BB54106D36546521BB7
:1055E000B341744607430C43A646CD07400849081B
:1055F000284392185B4105460D43EAD110461843F3
:1056000013D06046194650407140084306D06046AA
:10561000101AB34106D20122002306E00022012322
:10562000DB0702E00122D2435310009874460105C3
:10563000381C6141029C039D0019694100F07BF90F
:10564000BFE70000FD03000070B54B005B0803439B
:105650000BD04B005C0D002633466542B341D41796
:10566000AD1AA34102DB0020014670BD12053018BF
:10567000514170BDC217C10F504010B54018CA0744
:105680009623002100F01EF910BD10B500229623CC
:10569000114600F017F910BD0EB5C217C10F5040EA
:1056A000CA0740180021054B0293019200910A4657
:1056B0000B4600F04DF903B000BD000033040000BC
:1056C0000EB505490291002100910A460B46019151
:1056D00000F03EF903B000BD330400004100400279
:1056E0000122400AD205090E80187F2901DA002024
:1056F0007047962903DC9622511AC84070479639A4
:105700008840704770B5CD0F4A0009030123090B8B
:105710001B0519430B4BED070024520D9A4201DA89
:10572000002070BD074B34339A4203DC9A1A00F014
:105730009DF802E00449511888402C43F1D04042C2
:1057400070BD0000FF030000CDFBFFFF4A0009030E
:105750000123090B1B051943094B10B5520D9A4241
:1057600001DA002010BD064B34339A4203DC9A1A4A
:1057700000F07CF810BD03495118884010BD0000AE
:10578000FF030000CDFBFFFFC20FD207400040081F
:105790000BD0C10D0723DB01C91840020905400ADF
:1057A0001143C2084007114370470020014670476B
:1057B00010B5002904DB0124E40740428C41214656
:1057C000002B04DB1C460123DB075242A3418B4222
:1057D00000D1824210BD000010B5002904DB012475
:1057E000E40740428C412146002B04DB1C46012388
:1057F000DB075242A341994200D1904210BD000004
:10580000CB0FDB07490010B5490802460A4307D011
:105810000A0D07240903E401090B121B002A01DC0D
:10582000002010BDC900440F0C43C100E018D20590
:10583000801800F03FF810BD0122D207002800DBDD
:10584000101A002900DB511A8142704710B5202A36
:1058500004DB0146203A9140002010BD91402023F6
:105860009C1A0346E3401943904010BD10B5202A0E
:1058700004DB0846203AD040002110BD0B46D3403F
:10588000D0402024A21A91400843194610BD10B5FB
:10589000202A06DBCB170846203A1041C1170B43DC
:1058A00006E00B461341D0402024A21A9140084341
:1058B000194610BD002904DA401C490001D14008F6
:1058C0004000704770B40024050C05D1102400047A
:1058D00002D1002921D01124050E01D10002083483
:1058E000050F01D10001241D850F01D18000A41CEA
:1058F000002801DB4000641C002908D020252E1B55
:105900000D46F540A14000D001212943084301067E
:105910001B1B000ADB1D02D5002070BC7047DB0595
:10592000181880180029F8DA401C4900F5D170BC1D
:1059300040084000704710B5002B08DA0024401CD6
:10594000614192185B411A4301D14008400010BDEB
:10595000F0B51FB482B005460C0003D0084604F031
:1059600053FF02E004F050FF203002460090214631
:105970002846FFF76BFF049B059A04460F46184321
:105980001143084314D0184610431BD000984021FF
:105990000A1A18460599FFF769FF05460E46009A50
:1059A00005990498FFF752FF084305D0012004E051
:1059B0002046394607B0F0BD0020C11705430E430D
:1059C0002C43374300990E986305401A7905E40A81
:1059D00000220C43FD0A0A3002D500200146E9E707
:1059E0000105101969410C9C0D9D00196941FFF7D3
:1059F000A2FFDFE7FEB500231A461B1A8A4103DB2C
:105A00000020014603B0F0BD4A000D0301212D0B1B
:105A10000905520D0D43D10702D100186D41521EE8
:105A20005110FF31FF310131002704463E46384610
:105A3000009701910246012100200905FFF716FF9A
:105A4000C3197141F818324684468E464A41614670
:105A50002846611A904104D36046241A954176463F
:105A60001F46241900986D41401C00903428E1DD48
:105A7000F91930467041091BA84103D20022D243D4
:105A8000134601E00022134601980105381C7141BC
:105A9000FFF751FFB6E70000064C0125064E05E072
:105AA000E36807CC2B430C3C98471034B442F7D33F
:105AB000FFF70AFB00C9000820C9000870B58C1860
:105AC0000578401C6B075B0F01D10378401C2A113D
:105AD00006D10278401C03E006780E70401C491C79
:105AE0005B1EF9D12B0705D40023521E0DD40B7079
:105AF000491CFAE70378401CCB1A921C03E01D787E
:105B00000D70491C5B1C521EF9D5A142D8D3002050
:105B100070BD000038B50446064805490068FFF727
:105B2000E7FA604300E0401E00900028FBD138BD3A
:105B300040420F0084010020F8B5044600688168E7
:105B40008907890F012902D10168C90722D181681B
:105B5000114A10261140012500290ED181682943E0
:105B600081600120FFF7D6FF01F028F807460CE01E
:105B700001F024F8C01B0A2807D9606D3043606526
:105B8000A06D2843A0650120F8BD20680068C043CF
:105B9000C007EDD10020F8BD170000801FB50B48ED
:105BA00000900B4801900B4802900B480390694607
:105BB0000A4805F01FFA0A4A08481146083905F054
:105BC00007F900F06FFA002004B010BD0DC70008FF
:105BD000E9C6000849C7000847C70008900100202F
:105BE0001000002010B500231A4603E0845CE3187F
:105BF0009BB2521C8A42F9D3D84380B210BD000038
:105C000010B5034800F096FD024800F093FD10BD6A
:105C1000981700205017002030B5446C1C252C40EC
:105C20000125A540046C6560046863608368102BDF
:105C3000036803D099600068C26030BD9A60006854
:105C4000C16030BD1449012048720A4602205E320C
:105C5000507203203C3A507204200E3A50720F48A2
:105C60000D4B0078087022310870203108770C49FC
:105C70005A1C0878587149789971233318715971F1
:105C8000203318775977107551751A461E321075E2
:105C90005175107651767047E81100203E010020C2
:105CA0006001002010B503F0F5FE202003F0B0FFE6
:105CB000012005F009FC002003F0AAFF044805F0CC
:105CC000A7FA044805F056FD002005F08BFD10BD35
:105CD0000001002083800000F8B503F0A7FF052035
:105CE0000121000700F056FF0025144C002800D0C9
:105CF0006560134E0221304600F04CFF002815D19C
:105D0000012020700F48808F00280ED00127BF028D
:105D100000223946304600F04AFF0A2004F0C8FF4E
:105D200001223946304600F042FF6560012000F054
:105D300069FE022000F066FEF8BD00007001002040
:105D400000040050E80D00207047000010B508491D
:105D500000224A6107494B684C1523434B604B684E
:105D6000082423434B60C009C001026010BD00003D
:105D7000E0170020002002407FB500250C460646B3
:105D8000039500F00FFEE009029003A9019600952B
:105D9000684600F09FFD002804D000F0D7FD0020E9
:105DA00004B070BD00F0D2FD0120F9E710B500236A
:105DB00002E0C45CCC545B1C9342FAD310BD0000DB
:105DC00010B5214A00219069C305204804D54169D6
:105DD000022319434161911593699B0505D54369D8
:105DE0000124234343616302194393695B0505D58D
:105DF0004369082423434361E301194393691B0565
:105E000005D543690424234343616302194393691D
:105E10009B0405D54369102423434361630219435E
:105E200093699B0304D5446920231C4344611943AF
:105E30009369DB0305D54369402423434361A002F2
:105E40000143916110BD000000200240E0170020D6
:105E500070B5054600F0B2FE0646184C0AE0681C14
:105E600008D0002D04D000F0A9FE801BA84201D963
:105E7000032070BDA069C007F1D1A069800701D5DA
:105E80000220A061A069C00511D4A06980050ED4CC
:105E9000A06940050BD4A069000508D4A06980045E
:105EA00005D4A069800302D4A069C00303D5FFF71D
:105EB00087FF012070BD002070BD0000002002405F
:105EC000F8B51746002605460C4600F06BFD09E0C4
:105ED00029460220226800F047FD002804D1241D35
:105EE0002D1D361DBE42F3D300F030FDBE4201D25F
:105EF0000020F8BD0120F8BD10B508490246002079
:105F0000054B497905E044001C5B944203D0401CDA
:105F1000C0B28842F7D310BD8C130020700000205F
:105F200010B500F03CFE10BD10B5094801F05CF85A
:105F300080B2FFF7C5FB074A074BFFF7A5FA00221F
:105F4000064BFFF709FBFFF701FC80B210BD000014
:105F500004160020F853E3A59B843E4000408F4088
:105F600070B50024204603F015FA47494748A200BF
:105F7000641CE4B28150142CF9D3464944480A7990
:105F800002754979417544490A7802764978417623
:105F90003F490520133148720A2005F0DBFB7D20C4
:105FA000400105F0F1FB3A49002213310C2005F0C5
:105FB000BBFC00210C2005F0C9FC384801F014F8A6
:105FC000344C0125223C2085AD0309E0334801F023
:105FD0000BF880B22085E18EFF392D39884206DB2F
:105FE000E18E80B28842F1D349198842EED802206E
:105FF00005F000FC002003F0CDF9294D00210F2011
:1060000005F028FB28422064F8D0206C411C38D0D1
:10601000400435D58122D20100210F2005F059FC22
:106020000021102005F016FB41061948490E0022F8
:10603000C73005F045FB164DC735687A05281FD1D6
:1060400002221549681DFFF7BDF8002818D1114834
:10605000AE7C66710422691C3630FFF78FF8294642
:106060001331084672000D466930FFF787F86079F2
:106070002946420005484838FFF780F80320207081
:1060800070BD04F035FC0000FFFF0100EC130020A0
:106090004912002092000020600100200416002018
:1060A00000D0272410B5144C144822461032114653
:1060B000083904F08DFE0022114BE168A068FFF75B
:1060C0004BFA104A104B05F0B1FD00220F4BFFF7C1
:1060D000D3F900220E4BFFF7D7F9FFF791FB2060B1
:1060E00000221346E168A068FFF762FB01D0206838
:1060F00010BD0020206010BD000000209001002095
:1061000000AA8F406C45D9CC955BC83F0000F03F9A
:1061100040A5E54010B5084800F096FA0A21064867
:1061200000F032FA044800F01DF9800503D502485A
:1061300000F01AF980B210BDA8150020F8B52F4D57
:1061400000220121284600F032FDFFF7E3FFFFF7B0
:106150009CFA2B4E3146FFF79BF82A4C0122A06097
:106160001146284600F023FD2749A06800258842F3
:106170003EDB2078254F002815D02570FFF7CAFF99
:10618000FFF783FA3146FFF783F8A060FFF7FCFAC8
:1061900000223B46FFF76AF900221D4BFFF774F916
:1061A000FFF72EFB6060A068FFF7EEFA00223B4687
:1061B000FFF75CF9174A184BFFF766F906460F46DA
:1061C0006068FFF7E1FA134A144B5242FFF75CF99B
:1061D00032463B46FFF7A6F8FFF712FB1049606016
:1061E000884201DD616004E0FF21C905C84200D397
:1061F00065606068FFF772FAC0B2F8BD0004005035
:1062000000401B44480000200000604000000C409B
:1062100000E064403333333333B33040CCCCEC3F15
:106220000000C842F8B5054604464035287C0026E3
:10623000012808D001202874206881688907890F07
:1062400001290ED101E00220F8BD0168C90708D07C
:10625000606D2021084360650126002028743046C7
:10626000F8BD616DFF220132914302221143616545
:10627000C1688907890F0091C16889088900C160D8
:106280002068816892071143816000F097FC0746FF
:106290000EE000F093FCC01B0A2809D9606D0221B2
:1062A0008843102108436065002028740120F8BD50
:1062B000206880680028ECDB2068C168009A1143E0
:1062C000C160606D80088000401C6065C5E700000B
:1062D000F8B506460D464036317C01290DD0012126
:1062E000317401688A68520709D5416D2022114333
:1062F0004165002030740120F8BD0220F8BD174B25
:106300006A68D80547109A42154C8A6A2B6812D0E1
:106310005B035B0B1A438A622968490305D5A168B0
:106320000143A1600A20FFF7F5FB2868800312D51E
:10633000A06838430EE05B035B0B9A438A622968CE
:10634000490302D5A1688143A1602868800302D572
:10635000A068B843A06000203074F8BD01100000B0
:1063600000270140406D70470068006C70470000D6
:1063700070B5040006D0606D264600254036002822
:1063800002D006E0012070BDA5653574204600F0FE
:10639000D3F8606DC00603D421688868400705D52E
:1063A000606D1021084360653574EBE7606DFF2276
:1063B0000132904302221043606588688207920F81
:1063C0005B48012A02D10A68D2072BD103236268F5
:1063D0009B079A4205D05B429A4202D05B009A42E8
:1063E00009D10A69920092080A6121680A69636802
:1063F0001A430A610CE00A69920092080A618168F6
:106400000F22920491438160816862681143816028
:106410002168CA6818239A43CA602168CA68A368B9
:106420001A43CA60816801225206914381608168E3
:10643000A28E52061143816020688168C90004D48D
:10644000816801221207114381602068C168394ABE
:106450001140C1602069E168022825D00020014375
:10646000204620300278037B52035B001A4311431D
:10647000226B1143A26992031143E269D2031143D3
:106480002268D3681943D160616A0A46FF3AC23A6A
:1064900005D0A26A11432268D3681943D1604278BB
:1064A0000121012A02D00BE00420D8E7007800285F
:1064B00023D0606D202210436065A06D0843A06565
:1064C000E06B012820681FD00169C90703D001696A
:1064D00049084900016120684169C908C900416152
:1064E00020684169A26B11434161A565606D800818
:1064F0008000401C6065002070BD2068C2680123D8
:106500001B041A43C260DBE70269FF239B009A4326
:10651000026120680269236CA66C1A43636C3343E2
:106520001A430261206802690A430261D3E700004E
:10653000002701401902FEFF10B586B00446142161
:106540006846FEF734FE0E492068884216D10D4891
:10655000416B421511434163C16A01221143C1627B
:10656000C06A694610400590022000900320019007
:10657000002002900520000700F050FA06B010BD80
:106580000024014000100240F8B504464069254649
:1065900040350E4608280BD02068C068C00709D0D7
:1065A000606D202108436065002028740120F8BD3B
:1065B000082700E00C2700F001FB009011E0701CA0
:1065C0000FD0002E05D000F0F9FA0099401AB04221
:1065D00007D9606D042108436065002028740320FA
:1065E000F8BD206800683842E9D0606D0121490299
:1065F000084360652068C16809058A0F0C21002ADC
:106600001BD12022125D002A17D10268120714D56F
:10661000826853070122002B08DB43688B434360E9
:10662000606D130298431043606506E0606D20239F
:1066300018436065A06D1043A065A069002801D1D2
:10664000206801600020F8BD70B504462168002074
:106650008968490721D425464035297C01291CD069
:1066600001212974E169012904D02046FFF764FA69
:10667000002811D1616D0A4A1140FF2201321143F5
:1066800061650021A165297422681C2111602168BF
:106690008A6804231A438A6070BD022070BD00001E
:1066A000FEF1FFFF30B5014620314A790023022A6E
:1066B00004D00422C2630B71012030BD026814684B
:1066C0000E25AC431460026814686408640014600A
:1066D000446C1C22144001221546006CA540456004
:1066E0004A7118460B7130BD70B500240146203147
:1066F0004A79022A03D00421C163012418E0026808
:1067000013680E25AB431360026813685B085B00D7
:106710001360436C1C221340012215469D40036CFC
:106720005D604A7100220A71816B002900D08847A0
:10673000204670BDF0B4016C0D6801680C68466CB1
:106740001C2304221E401746B7402F420ED0670775
:106750000CD50C68A40602D40C6894430C60416C00
:1067600019408A40016C4A60016B1AE00227B74069
:1067700002462F402032002F17D0A70715D50C68EE
:10678000A40605D40C680A25AC430C6001215171A4
:10679000446C02211C40036CA1405960002111711E
:1067A000C16A002918D0F0BC08470827B7402F421B
:1067B00012D0240710D50C680E25AC430C60446C35
:1067C00001211C400B46A340046C6360C1635171FE
:1067D00000211171416BE4E7F0BC704770B5040013
:1067E0003CD01F48256814212818FEF781FC800042
:1067F00060641C482064022120462030024641711A
:1068000029681948E3680140A0686669184323694C
:1068100033431843A3691843E3691843236A1843B1
:10682000084328600121A0688903884210D00D48E0
:106830008030836A656C1C210D400F26AE40B34347
:106840008362656C63680D40816AAB400B43836271
:106850000020E06301215171107170BD012070BDF5
:10686000F8FFFDBF000002400F80FFFFF8B50446AF
:106870008C46203001790025012909D001260671B6
:1068800041790027012905D0077102252846F8BD66
:106890000220F8BD02214171E763206801684908C0
:1068A0004900016061462046FFF7B6F9206B0028D9
:1068B0002068016801D00E2205E0042291430160A6
:1068C000206801680A221143016020680168314391
:1068D0000160DBE7F8B51A4E0546307C0F4601280B
:1068E00007D0012030741748FFF7B2FA010002D038
:1068F00021E00220F8BD0020C04338606C6814E03D
:106900002046FFF723FA0F48FFF7A2FA01460E4888
:10691000426808239A434260426843159A434260A2
:10692000002901D03C6006E08034A8686A68C00194
:106930008018A042E4D8002030740846F8BD00005A
:10694000E017002050C300000020024005484168C5
:10695000022211434160416801221143416000203D
:106960007047000000200240F8B50C4C1646207C11
:106970000F46012808D0012020740948FFF768FA63
:106980000025002802D006E00220F8BD65613E60C7
:106990000348FFF75DFA2574F8BD0000E0170020FA
:1069A00050C3000011484168C9070BD0EFF31081B4
:1069B00072B60F4AC2600F4AC26081F31088416804
:1069C000C9070ED1416889070DD5EFF3108172B662
:1069D000094A0261094A026181F310884068800710
:1069E00001D50120704700207047000000200240C0
:1069F000EFCDAB8905040302BFAE9D8C16151413B1
:106A00007047000010B504494A69024202D048614B
:106A1000FFF7F6FF10BD000000040140FCB50023A5
:106A20000124A2E027462A469F403A406FD04D6895
:106A3000012D05D0022D03D0112D01D0122D16D11C
:106A400085680326AC465D00AE46AE406546B5435C
:106A5000AC46CE687546AE4065462E4386604668B5
:106A60000D79BE43ED06ED0F9D4035434560C66888
:106A70005F000325BD40AE46AE4335468E68BE403E
:106A80002E43C6604E68022E01D0122E14D1DE08AD
:106A9000B60036180196366A5D07B446EE0E0F252D
:106AA000B54000966646AE43B4460D69009EB540BB
:106AB00066462E43019D2E6206687546AE430D79EB
:106AC000AD07AD0FBD40354305604D68ED004BD5BA
:106AD000294D6E6B26436E639E08284DB6007519CE
:106AE000AC46AD689E07360F0F27B740BD4305275C
:106AF0003F07B84201D1002715E0214FB84201D12C
:106B0000012710E01F4FB84202D102270BE02BE013
:106B10001D4FB84201D1032705E01C4FB84201D1F7
:106B2000052700E00627B7402F436546AF60184DA4
:106B30002E684F689643FF0300D516432E606E689B
:106B40004F689643BF0300D516436E60AE684F682A
:106B50009643FF0200D51643AE60EE684F68964339
:106B6000BF0200D51643EE605B1C0A681546DA408A
:106B700000D057E7FCBD00000010024000000140BB
:106B80000004005000080050000C0050001C005091
:106B9000000401400069084000D0012070474269AC
:106BA00013460B401B0491430B4383617047002A3B
:106BB00001D08161704781627047000001488068A0
:106BC0007047000078010020024881680278891827
:106BD000816070477801002010B5084800240168E2
:106BE000402211430160204600F00AF8002801D03D
:106BF000012401E000F042FA204610BD00200240CE
:106C000070B504460D4D7D202978C000FEF770FA5E
:106C100001460B480068FEF76BFA00F02BFF0028D6
:106C200009D1042C07D200222146401E00F04EFA62
:106C300000206C6070BD012070BD00007801002054
:106C40008401002070477047F8B502F0EFFF604CF8
:106C50000120E070208AFEF718FD01467F20C00564
:106C6000FEF716FB5B4D06462968FEF7B8FA28606A
:106C70000120A16AC005814201DA084603E03046DE
:106C8000FEF702FBA062FF21C9050025C84200D320
:106C9000A562607800280BD102214F48FFF77AFFE8
:106CA00002004E494E4817D00022FFF780FFE562F0
:106CB00002214948FFF76EFF4A4E002855D0E56291
:106CC000B08AFEF7E2FC434F3968FEF7B5FD5FD2AC
:106CD0004549012008705DE00122D1034048FFF7DB
:106CE00066FF208AFEF7D1FC01467F20C005FEF733
:106CF000CFFAE16AFEF773FA3C49E0628842D7DDD9
:106D000038480127F926403000900A213046FEF726
:106D1000EFF9002903D131493148FFF701F9022188
:106D20002D48FFF737FF002801D0002701E0002F92
:106D300012D102212848FFF72DFF00280CD104F0C2
:106D40003DFF00990120888005F094FC642003F049
:106D5000AFFF28492648C8600A2003F0A9FF304643
:106D6000761EF6B20028D0D1A2E7208AFEF78DFC6D
:106D700001467F20C005FEF78BFAE16AFEF72FFA85
:106D80001D49E06288429BDB1A491948C86097E7B1
:106D900015480570708F401EFEF76CFC3968FEF7D1
:106DA0004BFD06D82079002803D014490120087033
:106DB00001E012480570708FFEF767FC3968FEF736
:106DC0003BFD04D22079002801D004F0B9FEF8BDC3
:106DD0003C010020740100200004005000800000ED
:106DE00000000050E80D0020760000200000404028
:106DF0000400FA0500ED00E00000A040860000203D
:106E0000704770B5040010D0022025462035A873C5
:106E1000204601F043FDA87B032805D0204600F062
:106E2000B9F80020A873687370BD012070BD704769
:106E3000704710B5044600680168C943C90708D106
:106E40008168C943C90704D1012141602046FFF789
:106E5000FBFE20680168C943890708D48168C943DB
:106E6000890704D4022141602046FFF7EBFE206829
:106E70000168C943490708D48168C943490704D454
:106E800004214160204600F0F7F820680168C943FA
:106E9000090708D48168C943090704D4082141605F
:106EA0002046FFF7ADFF20680168C943C90608D432
:106EB0008168C943C90604D4102141602046FFF708
:106EC000C2FE20680168C943890608D48168C943A5
:106ED000890604D4202141602046FFF7A9FF2068DD
:106EE0000168C943490608D48168C943490604D4E6
:106EF000402141602046FFF79AFF10BDF8B504001D
:106F000005D025462035A87B002802D006E00120C8
:106F1000F8BD00206873204600F04EF80220A873E8
:106F20002068C26884466368012B01D10620824331
:106F300016486169814202D0072040038243002B3A
:106F400001D1D82082431248A66802401846304337
:106F5000676A266A3E433043A66A30431043002BDB
:106F600002D0012B04D005E02369E2691A4300E056
:106F7000E2681043054A914202D0A26911430843D6
:106F80006146C8600120A8730020F8BDFFFF000023
:106F9000F8F119FF10B500680549884207D1054886
:106FA000816B4900490881630D2000F073F810BD22
:106FB000007C00400010024010B50068084988427B
:106FC0000CD10848816BC204114381630022012166
:106FD0000D2000F07BF80D2000F06CF810BD0000D3
:106FE000007C0040001002400068C069704700004B
:106FF000F8B504460220254620351746A8731D48DB
:107000000268C3041A4302602068C2689B121A43D4
:10701000C2602068026901263243026122681020A2
:107020005060206881611021204601F0A7FC0328F0
:107030001FD0216808204860206847610821204649
:1070400001F09CFC032814D0204601F027FCA87B0B
:1070500003280ED02068816831438160206801696F
:107060003143016120680169042211430161AE735B
:107070000020F8BD00040140704700000448416B47
:10708000012211434163816B020411438163704704
:1070900000100240002809DBC106C90E012088400B
:1070A00003490860BFF34F8FBFF36F8F7047000035
:1070B00080E100E0002805DBC106C90E0120884000
:1070C000014908607047000000E100E010B503F0DE
:1070D000EDFB10BD02494A6882434A6070470000D8
:1070E000007000400248016882151143016070473A
:1070F0000070004002494A6802434A60704700003D
:1071000000700040054801680222114301600448F4
:10711000016904221143016130BF704700700040D3
:1071200000ED00E0F0B5154A1368154D54152D6AB1
:107130002340ED07ED0F002B04D0002D02D0166880
:10714000A64316601668B608B600064316600D48DA
:10715000076904263743076101290DD040BF20BFCE
:1071600020BF0169B1430161002B04D0002D02D082
:10717000106820431060F0BD30BFF2E7007000409F
:107180000000014000ED00E0F8B50446007800275B
:10719000534D800671D5524E403EB06BC00004D4B2
:1071A000B06BA9050843B06301274E480168C905C3
:1071B00011D40168821511430160FFF7FFFC0090B4
:1071C00005E0FFF7FBFC0099401A642837D84548D2
:1071D0000068C005F5D532680321090560680A40DA
:1071E0000140914208D08103890F032904D13168FD
:1071F000890301D50120F8BD2A69032109040A4049
:1072000022D0084090421FD0207880061CD52869E3
:107210002A6988430121C9040A432A612A698A43E9
:107220002A612861C0050FD5FFF7C8FC009008E06F
:10723000FFF7C4FC0099411A2B48814201D9032071
:10724000F8BD28698005F3D561688803800F03289D
:1072500005D132680005824301400A433260286943
:10726000032261681204114008432861002F04D0F2
:10727000B16B012000078143B1632078C00705D0BE
:10728000E868A168800880000843E86020788007EB
:1072900005D5E8680C218843E1680843E860207858
:1072A000400706D5E868032189028843216908431D
:1072B000E8602078000706D5E868032109038843C1
:1072C00061690843E8602078000606D5E868032174
:1072D00089048843A1690843E8600020F8BD0000E4
:1072E000401002400070004088130000F8B50E46C0
:1072F000050038D05E480068C007C00FB04214D205
:107300005B4C20684008400030432060FFF756FC8B
:10731000074605E0FFF752FCC11B564881427AD868
:107320002068C007C00FB042F4D12878524C8007C3
:1073300005D5E068F0218843A9680843E060287813
:10734000C00752D06868022806D0032807D02168F9
:1073500001280AD0890504E02168890301E0216839
:107360008901002903DB0120F8BD4907F9E7E1683D
:10737000890889000143E160FFF720FC074668683F
:1073800002280AD0032814D001281ED029E0FFF7D4
:1073900015FCC11B374881423DD8E0680007800FCB
:1073A0000228F4D121E0FFF709FCC11B31488142DA
:1073B00031D8E0680007800F0328F4D115E0FFF70B
:1073C000FDFBC11B2B48814225D8E0680007800FD8
:1073D0000128F4D109E0FFF7F1FBC11B25488142E8
:1073E00019D8E0680007800FF5D121480168C90766
:1073F000C90FB14217D901684908490031430160FA
:10740000FFF7DCFB074608E005E0FFF7D7FBC11BF1
:107410001848814201D90320F8BD15480068C0070B
:10742000C00FB042F1D12878400706D5E0680721A7
:1074300009028843E9680843E0602878000707D517
:10744000E0680721C90288432969C9000843E06050
:1074500000F03AF8E168094A0906090F515CC84092
:107460000749086007480068FFF7CAFBF8BD00003D
:107470000020024088130000001002404EC800089F
:10748000840100207C010020044805490068C96887
:10749000044A4905490F515CC840704784010020E7
:1074A0000010024067C80008044805490068C96820
:1074B000044A8904490F515CC84070478401002088
:1074C0000010024067C8000870B51A4AD3681A490C
:1074D0000C2018408D0004280CD04E00082810D035
:1074E0000C2810D050680004410F0120C003491C33
:1074F000884070BD1068C00601D5084670BD28469A
:1075000070BD304670BD98020C4C000F205C1B0211
:107510009C0FD368641CDB0301D5314603E012687D
:10752000D20600D4294603F086F922460023FDF74F
:10753000F5FD70BD0010024000093D005EC8000866
:10754000FEB505007ED0FE4CE7680C20E6680740DB
:107550000120000406402878C00747D0082F05D036
:107560000C2F0AD101200004864206D12068800336
:107570003CD568680028E5D038E00120696800043F
:10758000814203D121680143216011E005230122DA
:107590001B0492049942216802D111432160F1E752
:1075A0008143216021680140009120689043206060
:1075B000686800280DD0FFF701FB009005E0FFF799
:1075C000FDFA0099401A64287BD820688003F6D51C
:1075D0000CE0FFF7F3FA009005E0FFF7EFFA0099EF
:1075E000401A6428F0D820688003F6D428788007F1
:1075F00056D50923E868042F0DD00C2F01D1002E99
:1076000009D000283CD02168994301432160FFF74D
:10761000D5FA064628E02168490701D5002891D00F
:1076200061681F22120291432A69120211436160AC
:107630002168994301432160FFF746FFE16809068D
:107640000A0F00E08BE1BF49895CC840BE49086071
:10765000BE480068FFF7D4FA002873D120E0FFF796
:10766000ADFA801B0228AFD820684007F7D56068C4
:107670001F210902884329690902084360600FE05D
:107680002068400840002060FFF798FA064604E0B2
:10769000FFF794FA801B022896D820684007F7D499
:1076A0002878C00660D5002F0CD0A86900284AD0E1
:1076B0002068FF21013108432060FFF77FFA06466A
:1076C0002EE0C1E02068800502D5A8690028A6D078
:1076D0006068072149038843296A0843606060683D
:1076E000297F0002000A090608436060286A410BEE
:1076F0000120C003491C8840E16809060A0F91492E
:10770000895CC8409049086090480068FFF778FAA3
:10771000002817D128E0FFF751FA801B0228A2D8D1
:1077200020688005F7D56068072149038843296AE6
:10773000084360606068297F0002000A0906084368
:10774000606011E0E2E02168FF20013081432160A8
:10775000FFF734FA064604E0FFF730FA801B0228F0
:1077600072D820688005F7D42878794E000724D590
:1077700068690028306910D0012108433061FFF7A3
:107780001DFA009005E0FFF719FA0099401A022847
:107790005AD830698007F6D50FE0400840003061C4
:1077A000FFF70CFA009005E0FFF708FA0099401A7D
:1077B000022849D830698007F6D42878400766D572
:1077C00000200290A06BC00006D4A06B0121090725
:1077D0000843A063012002905E480168C90511D4E6
:1077E0000168821511430160FFF7E8F9009005E098
:1077F000FFF7E4F90099401A642825D85548006835
:10780000C005F5D5FF20AA680130824203D1316955
:107810000143316111E001218902002A07D00523CB
:107820001B029A4203D132690A433261EFE732699F
:1078300082433261306988433061A868002810D0E3
:10784000FFF7BCF9009008E05FE0FFF7B7F90146E9
:107850000098091A4048814257D830698005F4D50C
:107860000DE0FFF7ABF9009006E0FFF7A7F90099EC
:10787000411A3948814248D830698005F5D40298C8
:10788000002804D0A06B012109078843A063686A1F
:10789000002866D00C2F3ED001263606022820682C
:1078A00005D0B0432060FFF789F905462FE0B043CB
:1078B0002060FFF783F9074604E0FFF77FF9C01B5C
:1078C000022822D820688001F7D4E96AA86AE26811
:1078D0000843296BFD231B049A4311430843E060CE
:1078E000206830432060FFF769F9054604E0FFF7A0
:1078F00065F9401B022808D820688001F7D530E0E0
:10790000FFF75CF9401B022801D90320FEBD206867
:107910008001F5D425E00128F8D0E06801210904B0
:10792000AA6A014091421AD10F218904EA6A0140F2
:10793000914214D1032189050840296B88420DE04A
:10794000001002404EC80008840100207C01002085
:1079500040100240007000408813000001D0012058
:10796000FEBD0020FEBDF8B504000ED0FF27606A02
:107970000537002500280AD0256165612646403676
:10798000A562707C002807D00AE00120F8BD60687D
:10799000B842F3D0E561F1E73574204600F03EF8D7
:1079A000022171742068026840239A4302602123F7
:1079B000A26860689B021A4038401043E3688A025C
:1079C0001340184323690B40217D1843C907C90F91
:1079D0000843A169931019400843E169382319400D
:1079E0000843216A802319400843A16A9300194083
:1079F000084321680860A0690421000C0840616AFE
:107A0000102319400843216848602068C1699143E8
:107A1000C1616565012070740020F8BD10B586B0A5
:107A2000044614216846FDF7C2FB104920688842CD
:107A300019D10F48416B821411434163C16A01227D
:107A40001143C162C06A002110400590E0200090FF
:107A500002200190032003900291049105206946C1
:107A60000007FEF7DBFF06B010BD0000003001404C
:107A700000100240094910B5401E884201D901207A
:107A800010BD074C60610321081F02F00FFF0020AA
:107A9000A06107202061002010BD0000FFFFFF0053
:107AA00000E000E0F0B502462032137E012B1ED02C
:107AB000012515760223537606687468B36870272B
:107AC000BC430F68274377600068AC07A04205D02D
:107AD000084CA04202D0084CA04204D1802449683E
:107AE000A34319438160557600201076F0BD022033
:107AF000F0BD0000000801400014014070B5050011
:107B000005D02C462034607E002802D006E00120FB
:107B100070BD00202076284600F010F80220607624
:107B2000291D286802F0F8F80120A077A076E076F9
:107B3000207760776076002070BD0000006801212A
:107B40008907884204D10348816B01221143816374
:107B50007047000000100240F8B505460446203585
:107B6000287E012817D001262E760220687622680A
:107B700090687727FF23B8431B02984390600A68F8
:107B8000502A31D00EDC202A4BD006DC002A48D007
:107B9000102A3AD145E00220F8BD302A41D0402ACF
:107BA00033D136E0602A27D0702A12D0012000039A
:107BB000121A2AD0824228D1CB684A688968206884
:107BC00002F0E3F82068816801229203114381608A
:107BD0001BE0CB684A688968206802F0D6F8216803
:107BE00088683843886010E0CA684968206802F0F5
:107BF00046F95021206806E0CA684968206802F00A
:107C00004FF96021206802F0CBF86E7600202876CC
:107C1000F8BDCA684968206802F031F9402120683F
:107C2000F1E711462068EEE710B586B0044614214E
:107C30006846FDF7BCFA012120688907884212D105
:107C40000A49CA6A02200243CA62C96A0190014015
:107C5000059141020091002102910391049069462F
:107C60000348FEF7DBFE06B010BD00000010024026
:107C700000040050F8B5064604462036307E0D4616
:107C800001280BD0012008273076002A08D0042ACA
:107C900016D0082A2AD00C2A4DD137E00220F8BD90
:107CA000206802F085F82068816939438161206885
:107CB000816904229143816120688169EA6812E048
:107CC000206802F08DF8206881690122D2021143F8
:107CD000816120688269012189028A43826120686A
:107CE0008169EA6812021143816124E0206802F090
:107CF00090F82068C1693943C1612068C1690422D4
:107D00009143C1612068C169EA6812E0206802F00D
:107D10009BF82068C1690122D2021143C161206829
:107D2000C269012189028A43C2612068C169EA6887
:107D300012021143C16100203076F8BD70B5050014
:107D400005D02C462034607E002802D006E00120B9
:107D500070BD00202076284600F00FF802206076E3
:107D6000291D286801F0D8FF0120A077A076E076D1
:107D7000207760776076002070BD704770B505464B
:107D80002C4602202034002908D004290BD00829D1
:107D90000ED0627F012A10D0012070BDA27E012A80
:107DA000FAD1A0760AE0E27E012AF5D1E07605E07C
:107DB000227F012AF0D1207700E060770122286835
:107DC00001F0D6FF0122286892070121904205D0D8
:107DD000074A904202D0074A904204D18268520773
:107DE000520F062A02D002680A430260002070BDCA
:107DF000000801400014014070B504460D460068BB
:107E0000002201F0B5FF2068016A0C4A114203D13B
:107E1000016849084900016001202034002D06D086
:107E2000042D06D0082D06D06077002070BDA07606
:107E3000FBE7E076F9E72077F7E700001111000093
:107E40007047704770470000F8B502680446D06973
:107E500011689668814B05461D402023002D6CD08B
:107E6000F7077F4DFF0FBC460D402F4379D02546C5
:107E7000C7078035002F06D0CF0504D5012717622C
:107E80002A683A432A60820708D5F20706D0276895
:107E900002223A622A6804273A432A60420708D538
:107EA000F20706D02668042232622A68022632438C
:107EB0002A6002070AD50A461A406646324305D0B0
:107EC0002668082232622E6816432E60020508D505
:107ED0004A0106D501222668D20232622A681A4374
:107EE0002A602A68002A30D0800606D5880604D584
:107EF000616E002901D0204688472868216889687A
:107F0000490602D42821084225D0204602F0DFF994
:107F100020688168490619D5826840218A438260B9
:107F2000206F002812D04F498163206FFEF7DCFBE1
:107F300000280AD0206F816B06E0850611D58D06DA
:107F40000FD5616E77E020468847F8BD2046FFF7E1
:107F500079FFF8BD05E02046FFF774FF0020286098
:107F6000F7E7256E012D56D1C50654D5CD0652D55D
:107F7000102616622068816825464906403500298A
:107F80002ADA226F116849680904090CE1D02F8BA5
:107F90008F42DED9698311680968890617D40168A0
:107FA000320191430160206881684908490081607D
:107FB00020688168402291438160E3670020206649
:107FC00020680168B1430160206FFEF76BFB288BCE
:107FD000698B401A81B21AE0298B6A8B891A6A8BE5
:107FE00089B2002AB5D00029B3D00268FF25213517
:107FF000AA43026020688268520852008260E367E8
:1080000000202066606620680268B2430260204655
:10801000FFF716FF9DE7C50208D5750206D50120BA
:10802000000510622046FFF70CFF92E7050605D514
:108030000D0603D5A16E002985D18AE7400688D5B3
:10804000480686D5116820464024A1431160836705
:108050000021816600F043F97BE700000F08000073
:1080600020010004F5A1000810B5040003D0A06FA2
:10807000002802D007E0012010BD00217420015526
:10808000204600F027F82420A067206801684908EE
:1080900049000160204602F06DF90128ECD0606AC9
:1080A000002802D0204601F08FFF20684168092295
:1080B000D20291434160206881682A229143816005
:1080C00020680168012211430160204601F0E2FFAF
:1080D00010BD0000F0B587B0064614216846FDF7D4
:1080E00066F82C493068884251D12B48416B0122F7
:1080F000920311434163C16A01221143C162C06A04
:108100000025104005900320400200900220032724
:1081100001A9A1C104200490052069460007FEF7CB
:108120007DFC1F4C1D48A560E56081C48027E5608B
:10813000A7602020256160610002A0611848083C0A
:10814000FEF74CFB002801D0FDF7FEFD3467A66268
:10815000144C12482146143820600320606010201F
:108160000831A1C16561A561E56120462562FEF780
:1081700035FB002801D0FDF7E7FDF4660022012160
:108180001B20A662FEF7A2FF1B20FEF793FF07B09D
:10819000F0BD0000003801400010024030000240F5
:1081A000501700209817002070B5C36F202B27D1DF
:1081B00000290BD0002A09D0012483682403A3429C
:1081C00006D10369002B03D1CB0701D0012070BD7C
:1081D000034660331C7D012C12D001241C75002342
:1081E0000366084C0368A34207D05C68240204D5E8
:1081F0001C680125AD062C431C6002F0BBF970BD64
:10820000022070BD0048004070477047FFB504462B
:10821000806F83B017460D4620285ED1002D0AD00E
:10822000002F08D0A168C001814207D12069002831
:1082300004D1E80702D0012007B0F0BD204660302D
:108240000090007D012848D0009801210175002090
:10825000802108512120A067FEF7B0FC2646403659
:108260000190378277820120A1680003814202D108
:108270002069002805D02F460025009900200875A8
:1082800011E00027F9E700228021204602F0B8F92A
:10829000002815D1002F15D02168387888627F1CFE
:1082A000708A401E7082708A019B00280698009098
:1082B000E9D100224021204602F0A2F9002808D08E
:1082C0000320B9E728882168C005C00D8862AD1C6D
:1082D000E6E72020A0670020AEE70220ACE7704769
:1082E000034D044C04A002F085FAE560FAE70000B3
:1082F0000400FA0500ED00E0486172644661756CA7
:10830000745F48616E646C65722E0D0A0000000097
:1083100000B585B014216846FCF749FF04490220E6
:10832000C8800449488300F053FC05B000BD00003C
:10833000280E00203C01002010B50524240700224F
:1083400004212046FEF733FC002208212046FEF7D8
:108350002EFC0A2002F0B3FC012204212046FEF785
:1083600026FC0A2002F0ABFC002204212046FEF786
:108370001EFC10BD10B50524240700220421204650
:10838000FEF715FC012208212046FEF710FC0A200A
:1083900002F095FC012204212046FEF708FC0A2089
:1083A00002F08DFC002204212046FEF700FC10BDE7
:1083B000F8B5002405260746254636070022042185
:1083C0003046FEF7F4FB0A2002F079FC012204217A
:1083D0003046FEF7ECFB6006040E08213046FEF73F
:1083E000D9FB002801D0641CE4B2052002F067FC30
:1083F0006D1CEDB2082DE1D3002F03D0FFF79CFFD9
:108400002046F8BDFFF7B6FFFAE770B5052605462A
:108410003607002204213046FEF7C9FB0024E80994
:1084200001D0012200E0002208213046FEF7BFFB08
:108430006806050E0A2002F042FC012204213046A3
:10844000FEF7B5FB0A2002F03AFC00220421304678
:10845000FEF7ADFB0A2002F032FC641CE4B2082CEB
:10846000DDD370BD10B50524240701220821204664
:10847000FEF79DFB012204212046FEF798FB002217
:1084800008212046FEF793FB0A2002F018FC002288
:1084900004212046FEF78BFB10BD10B505242407F0
:1084A000002204212046FEF782FB002208212046FC
:1084B000FEF77DFB0A2002F002FC01220421204687
:1084C000FEF775FB012208212046FEF770FB0A200B
:1084D00002F0F5FB10BD70B505252D070024012223
:1084E00008212846FEF763FB062002F0E8FB012284
:1084F00004212846FEF75BFB062002F0E0FB07E0C4
:10850000641CE4B2FA2C03D9FFF7C7FF012070BD49
:1085100008212846FEF73EFB0028F1D10022042165
:108520002846FEF744FB002070BD0000F8B501F0BE
:10853000E3FD01F013FE5B480068C069FDF7F4FC41
:10854000594C5A49A082898F594E0025002931D0B3
:10855000A26A730357499A4202DB02220A7000E0C2
:108560000D700A7801218902002A05D0012A0ED057
:10857000022A10D0032A1DD1608B01282ED0022898
:1085800018D1484808214038FFF736FC12E0FF2296
:10859000F5329042F0D2608B01281DD0022804D021
:1085A00008E03046FEF703FB04E03E48082140386F
:1085B000FFF7E4FBFDF7C2FD20700121C902304640
:1085C000FEF7E8FA0127FF0300282DD03A4805609E
:1085D000A079002804D007E00022E2E70122E0E7CA
:1085E0000120A07102F06EF880213046FEF7D2FA29
:1085F000002806D0002208213046FEF7D8FA0122D2
:1086000005E0012208213046FEF7D1FA00220520BC
:1086100039460007FEF7CBFA244C284E4034A08C94
:10862000274F012803D01CE0A5710022EAE7254866
:108630006946088072B680212348FDF79DFB00281B
:1086400004D0022269462048FDF73AFC62B61FA01A
:1086500002F0D0F8A58404F00DF8642002F028FBA5
:10866000FE60608C012808D110486584058004F004
:1086700001F8642002F01CFBFE60208C012806D16A
:10868000258403F0F7FF642002F012FBFE60074828
:10869000124A0188914202D1C088002800D1FE60B0
:1086A000F8BD0000CC1600203C010020E80D0020A1
:1086B0000004005084000020740100200400FA052A
:1086C00000ED00E0AAAA0000384A0008BDF8C8EB97
:1086D000C9FDBCB6C4A3CABD0D0A0000AA5500005E
:1086E00038B500246946202000F0AAF868460078D2
:1086F000572800D001246946212000F0A1F86846DF
:108700000078032800D001246946222000F098F860
:1087100068460078402800D001246946232000F0F4
:108720008FF868460078082800D001246946302078
:1087300000F086F868460078AA2800D0012469462F
:10874000322000F07DF80C486946008F0978884295
:1087500000D001246946332000F072F806486946CB
:10876000403040880978884201D1002C02D0044969
:108770000248C86038BD0000E80D00200400FA057A
:1087800000ED00E038B55721202000F07AF80321F1
:10879000212000F076F84021222000F072F8082114
:1087A000232000F06EF8AA21302000F06AF810486B
:1087B000018F142901D8002901D1012101870C4C16
:1087C00040346188142901D8002901D10221618037
:1087D000008FC1B2322000F054F8A178332000F0AD
:1087E00050F8684600F006F80A2002F068FA38BD32
:1087F000E80D002010B501460F2000F021F80028F8
:1088000000D0012010BD10B50446FFF72BFE32202A
:10881000FFF7FBFDFFF75FFEE0B2FFF7F6FDFFF7A6
:108820005AFEFFF71FFE3320FFF7EFFDFFF753FE61
:108830000020FFF7BDFD0446FFF72FFE204610BDC8
:1088400010B50C46FFF7DFFF2070012010BD70B59A
:108850000D460446FFF706FE3220FFF7D6FDFFF770
:108860003AFEE0B2FFF7D1FDFFF735FE2846FFF7ED
:10887000CCFDFFF730FEFFF710FE0A2002F01FFAD2
:1088800070BD10B5FFF7E3FF012010BD10B5024821
:10889000FEF7CFFA10BD000004160020FEB5044616
:1088A000002772B6334A01688B1804D13248C76872
:1088B00003208004074088680190C86800904869D8
:1088C0008E69002B08D12C4940398B6ACD042B438B
:1088D0008B628B6AAB438B62014631433CD02549A6
:1088E0002368CB4205D12449CA6803239B049A43D9
:1088F000CA6025462035002810D021680A69012366
:108900001A430A61216848610821204600F036F8C0
:10891000032800D1A873216808204860002E10D0D9
:1089200020680169012211430161206886611021DC
:10893000204600F023F8032800D1A87321681020F6
:1089400048600C482168C14206D10B48C168032227
:10895000920491433943C160206801694908490084
:10896000016121680198886021680098C86062B63A
:10897000FEBD00000084FFBF4010024070B50646F7
:108980000B480D46002409490068FCF7B1FB7D2126
:10899000C90048433168401E00D103240B682A46B1
:1089A0009A4301D00028F6D1204670BD204E000029
:1089B000840100201CB5002116480091144A019141
:1089C0000260C16312054260816007228263012256
:1089D00002610246C16020321170FF235170C23320
:1089E00043628162117301638161042241634261C8
:1089F000C161FDF7BDFC08480090801301906946F5
:108A00000448FDF765FC00210248FDF70BFC1CBD86
:108A100000240140A81500200200000408B5084801
:108A2000016B012211430163006B01211040009092
:108A300000220A20FEF74AFB0A20FEF73BFB08BD96
:108A400000100240F0B587B014216846FCF7AFFB78
:108A50004748C26A04210A43C262C26A0A400592B8
:108A6000C16A80263143C162C16A31400591C16A41
:108A700001242143C162C16A21400591C16A0225D6
:108A80002943C162C06A22462840059005201C2166
:108A90000007FEF78CF8012236493748FEF787F8C1
:108AA000002236493448FEF782F891210520002241
:108AB00009020007FEF77BF83148019000270520E6
:108AC0006946029700940007FDF7A8FF0C2000906C
:108AD00011200190032003900520029769460007AA
:108AE000FDF79CFF10206A46039591C20520694658
:108AF0000007FDF793FF1120019002976946039745
:108B000000941D48FDF78AFF1E48019069460095B4
:108B100002941948FDF782FFE00200906946019730
:108B200002951548FDF77AFF1748694691C16946D5
:108B300011480397FDF772FF91200002694691C129
:108B40000520694600070397FDF768FF69460A4854
:108B5000019700960294FDF761FF00220121052094
:108B6000FEF7B4FA0520FEF7A5FA07B0F0BD000045
:108B70000010024001020000000400500830000014
:108B800000001110000021100832000010B50F4C39
:108B90000D482060FF20053060600020A060E0608C
:108BA00020616061E0610121206249026062A1618F
:108BB000A0620720E0622046FEF7D5FE206801682B
:108BC00040221143016010BD0030014034160020E6
:108BD00010B58AB000240494059406940794089470
:108BE0000121184809940094019402948907039480
:108BF0000160092184604160046113494461C160DE
:108C0000FEF77CFF01200003049004A90D48FEF745
:108C1000A3FF0C48FFF792F8089408A909480994A3
:108C2000FEF740FF6020009008480190029408225F
:108C3000694603940348FFF71DF80248FEF7F4FF66
:108C40000AB010BD8C1600209304000057020000EB
:108C500000B585B014216846FCF7A9FA0E480D4905
:108C60000160E1214902416000218160C160016130
:108C700081610C22C16142610162302141620121A6
:108C8000090381634900C163FFF7EEF901F014FDA8
:108C900005B000BD00380140CC1600207047000030
:108CA000F0B589B00A2002F055FD7D20400102F0A8
:108CB0006BFDFF4C0025A570FE482066607C0C28EB
:108CC00001D30B20607460790A2801D90A206071F1
:108CD000F948E570F94E00783071F949A0790978C2
:108CE00040000843A17D89000843F071E06BF070FB
:108CF000010A3172401CE0636079B0744200304672
:108D0000F0491330FCF73AFA6079EE4982004000EE
:108D1000801960311330121DFCF730FA607906219A
:108D2000420048438019E8491730921CFCF726FAA4
:108D30002E20205E002803D0E449098A0818E08527
:108D40006079DB49C000223182190B7B53764B7B63
:108D5000937606227272DE4A1D301278B272A28CAD
:108D60003273D64A0B79133A13754979517500223B
:108D7000D24902F0D9FD60790021C0001D3002F017
:108D8000E5FDD448FEF730F901272085BF0309E04F
:108D9000D048FEF729F980B22085E18EFF392D39C0
:108DA000884206DBE18E80B28842F1D3C91988423D
:108DB000EED8022002F01EFDC0480126C571A57440
:108DC000A5732674E573C348FEF70EF96085074660
:108DD000E5706079FCF774FCBF4AC04BFCF754FBAC
:108DE00001F002FF0022BE4BFCF79CFAFCF7AEFC40
:108DF0000006C10CC81980B2F103A085884201D3D6
:108E0000401AA085B748E0642079401C2071B14821
:108E1000FEF7EAF82085AB48A54F64384037069046
:108E2000B1E1AC48FEF7E0F820850BE0A948FEF779
:108E3000DBF880B22085A18D884203D3AA4A891825
:108E4000884207D300210F2002F004FCA7492064C8
:108E50000842EBD0206C411C1FD040047ED58122FB
:108E6000D20100210F2002F034FD0021102002F079
:108E7000F1FB41069348490E00227C38E16502F07F
:108E80001FFC002002F080FC002002F032FC8D4824
:108E90007C38417A0729C3D101E001F029FD022283
:108EA0009349401DFCF78EF90028B9D102F09FFDCF
:108EB000E167A06702F088FD7D4B803303C3E07853
:108EC0008049401CE07083390B7A68460370497A08
:108ED000417000880390E18C88427DD177498548B4
:108EE0008C31C98E0180754971488C31098F41845C
:108EF0007848FEF779F8208502F0BEFA6C48FF2228
:108F000080300168406852040023891858410206E5
:108F1000080A10434108490000900A0E08026449FB
:108F20008031CA6088606548E36F0A30A26F02F042
:108F300033FD60798100614808185D491630803141
:108F40000CC902F029FD5A488030C36882685B482A
:108F5000123002F021FD0821584800E006E141727C
:108F6000B430C07C0009607514D0564802226049B4
:108F70007738FCF727F900280CD15048A674C67141
:108F8000E06D50491638C2B26639C81DE274FB3034
:108F9000FCF7F4F860790022800048491C3002F0A8
:108FA000C3FC6079002180001C3002F0CFFC0098E7
:108FB00002F0C9FB012002F01DFC207302214E4883
:108FC000FDF7E8FD00281DD000213D4801703B4918
:108FD0008C31488E049000E05AE03881888E788188
:108FE0008446A06CFF310531E0640860DC392065FF
:108FF000C97C0907090F032900D02175E16D1C29DF
:1090000002D015E00121E0E72C49294A8C31C98FB3
:109010001186069B2C4A1B881380884207DD002896
:1090200005DD002903D0207E401C207600E0257657
:109030002571A6730498B8816046F881E673608C48
:109040002E49FF30C33080B2608488420CD9494237
:109050004018608427487D220188D200491C89B2CB
:109060000180914200D3058022487D210088C900FB
:109070004843618C4018606500F074FD207B002837
:1090800005D100210F2002F0E5FA0006F9D583E0B2
:10909000FCF732FF0B4A03219032115407498C31FF
:1090A0004A8E3A81898E7981E26D1C2A2ED127E081
:1090B000700000203F420F003C0100205C120020A5
:1090C000700100208C130020C8140020280E0020FE
:1090D0004C01002004160020B81E85EB51B8CE3F8D
:1090E00000000840A0860100983A000000D0272424
:1090F000600100206C01002000040050E703000024
:10910000614B4200D318069A12885A8080005F4B48
:109110005E4AD43B02905D4982189B8F13803031A8
:109120004118A26C4A605A4940185A4916300CC975
:1091300002F032FC216EA06C884207DA534A029991
:109140005158012902D12066039905914F49029A8D
:109150008958814217DD012915DD2146002812DDDD
:109160000398C8840220087065730CE04A4A002105
:109170000F2002F0AEFB6079E178401C814202D002
:10918000002002F0B6FA208DA18D884200D248E678
:10919000424A89188842FAD8A07B012801D00220CF
:1091A000A07302F069F93C4A00210F2002F091FB04
:1091B0002079002817D03A4909888A008A18824203
:1091C00000D22570002000F0E5F8A07C002839D0FE
:1091D0002E496C310B78A372487860728A782272BB
:1091E000022B17D02EE0E16C226E323920468A42E3
:1091F0000EDAC1792A4A491CC9B2C17112885200DB
:109200008A42E2D20599C184022101706573DCE7CC
:10921000E571DAE710280CD0C82813D2214BC91CFD
:109220001818FBF7ABFF03F025FA642001F040FDAE
:1092300033E61D4D28684000000E03D1C878FCF7C6
:1092400024FA286000202378627B65790FE00F4EB6
:109250004100303E775A1836765AB74205D00B4F48
:10926000022300220126483F7E52401CC0B2A84281
:10927000EDD323706273084A002180320F2002F080
:1092800028FB09B0F0BD0000C8140020BC1300206A
:109290005C120020F000002000D02724983A000043
:1092A0004C010020E80D002064010020F8B52E4C90
:1092B0000546E06E2D4A281A411E2067914215D2BC
:1092C0001A21615E081AFCF7E7F9294A294BFCF7D5
:1092D000DBF8064632200F46205EFCF7DDF9324609
:1092E0003B46FCF71FF8FCF70DFA6086002060761D
:1092F0001D481C23C35E828C1F48008884461F487B
:1093000006881DE06046484380181D4F80B23880B3
:10931000302778436427643078431A4F6066C01959
:1093200085420BD2C8B2184932220880606EA25E14
:10933000411BC9188918A166E066F8BD491C617611
:10934000617EB142DED330204243104864211018C0
:1093500048430F494118E16660663221401B615E57
:10936000C0184018A066F8BD70000020CF070000AC
:109370009A9999999999B93F5A0100204C01002076
:109380006E01002078ECFFFF5801002074270000D8
:10939000C0BDF0FFFEB5294D2988491C8FB2284970
:1093A0002F800E88FCF778F9264A274BFCF76CF8DB
:1093B0000191009025483146FBF79AFE244C218FFD
:1093C0004218B74206D3002028802248019E101878
:1093D000009D02E01046019E009DFCF771F93346A6
:1093E0002A46FBF79FFFFCF7B1F9A086012580B262
:1093F000ED03A84201D3401BA086E08BFCF760F987
:10940000154A164BFCF7A8F80646A08E0F460090AA
:10941000FCF756F932463B46FBF784FFFCF796F91A
:1094200080B2E086A84201D3401BE0860C49009838
:109430000968486100982087FEBD0000580100209F
:109440004C0100201904560E2D624040E17A0000C4
:10945000700000201F050000F853E3A59B843E40E8
:109460000416002070470000F0B589B00020049079
:109470000A2002F06FF97D20400102F085F9B3481F
:1094800000228270C16BB34C491CC163B049C38DCB
:10949000098A2546C918C1852146C275133107912D
:1094A000473103916D393135AB4F22300591029030
:1094B000A64E0F21A948717100782071A84AB07991
:1094C000127840001043B27D92001043E071B08FDB
:1094D000E070000A2072A17431461E229C31079868
:1094E000FBF74CFE402228469E49FBF747FE0299B7
:1094F00003980A7BC274497B0175092060729A48FF
:109500000078A072B08C2073F07D410030469C3012
:10951000091805980A780275497841757620002265
:109520008C4902F001FA70790621484300211C3071
:1095300002F00CFA022002F05DF900210F2002F087
:1095400089F838423064F8D0306C411C18D040049F
:109550007ED58122D20100210F2002F0BAF900212C
:10956000102002F077F841067A48490E0022B43004
:1095700002F0A6F87748B430417A022902D0BDE063
:1095800001F0B6F902227949401DFBF71BFE0028C5
:10959000F5D16E480222C07D41006C489C3009180C
:1095A0006C48B530FBF70EFE0028E8D102F01FFA38
:1095B000664AD167906702F007FA644A803203C2B4
:1095C000049800282CD1012004906248684E8C3009
:1095D000C08E604930805D488C31098F4184654878
:1095E000FDF702FD5949644A0885488CFF30C330B5
:1095F00080B2488490420CD9524280184884308806
:109600005D4A401C80B20B323080904201D3002072
:10961000308030887D22D20050434A8C80184865C3
:109620004C4869468C30428E0A80808E4880494979
:109630000422B531C81FFF38FBF7A0FD4348494A53
:10964000C07D0099800011504049803103C900E07D
:1096500075E0FF235B040022C01851410906060A89
:109660000E43304602F06FF8710849000A0E0802F6
:10967000364900268031CA6088603448C36F826FE3
:109680003448483802F088F9304880300CC83148F6
:10969000443802F081F92D488030C36882682D4833
:1096A000403802F079F92B49002252393C2002F06F
:1096B0003BF900213C2002F049F9012002F09AF820
:1096C0002249087308468078401C887001210520D3
:1096D000C9030007FCF724FC1C48007B002805D1C7
:1096E00000210F2001F0B6FF0006F9D580220021ED
:1096F0000F2002F0EEF81548467002E013490120F1
:1097000048701248C17D491CC9B2C1750F2900D2E9
:10971000CEE60498002810D10C4A1849908C0028F5
:1097200002D00B88984201D908889084144980B2ED
:109730000988401E48431349088009B0F0BD124A09
:1097400000210F2002F0C5F8D8E7000070000020CB
:10975000280E00205C12002000D027243C010020AD
:1097600070010020781400204C01002060010020CE
:109770006C01002004160020E703000048010020CF
:10978000460100204401002000902724F8B531490B
:109790002F48086002F012FA2F4800F0A3F92F4C6E
:1097A000E0822D48801C00F09DF920832A48001D8E
:1097B00000F098F960832B482949418001464031E7
:1097C0000979294F0906090E617006D1C780012168
:1097D000C1870A21418700218187244AC18E1170E7
:1097E000C18F2171818F6171817AA1708588052176
:1097F00065626181C6883046FBF77AFCA08101462C
:109800002846FBF775FC8800081885B216482581A4
:109810006843FBF755FF164A164BFBF79DFEFBF717
:1098200095FFE081658231463846FBF761FC208276
:109830000146C820FBF75CFCE0830120A083FCF715
:1098400073FBA082E2890C490C48FDF7D1FBF8BDFF
:10985000E5A6000868000020004F00083C01002039
:109860002E020000E80D0020E80300001800002090
:10987000F853E3A59B843E40FF7F000004160020C0
:10988000F8B5754C00202071744D01202880744E6D
:10989000C8203080E07A401CE072C00706D0A08C5F
:1098A000411EA184022801D2C820A0840120C04307
:1098B000FFF770FD0A2001F04DFF7D20400101F00F
:1098C00063FF02216748FDF765F900283FD00020BB
:1098D000654980000978664F490008436349097863
:1098E0000843B872102078726248C1887D20C00099
:1098F000FBF7FEFB787360485E490078B873384622
:109900000B308A780270C97841705A49421C203164
:109910000B7ED370497E11715649D01C22310B7ECB
:109920005371497E9171534940310A7C0271497CDF
:10993000417100223946172001F0F6FF002117205F
:1099400002F004F8022001F055FF4C4F03E0012023
:10995000BEE7FEF7EBFD00210F2001F07BFE384251
:109960002064F6D0206C411C73D040046FD5812256
:10997000D20100210F2001F0ACFF0021102001F0E6
:1099800069FE41063A48490E0022B430E16501F013
:1099900097FE374FB437787A112858D102223849C8
:1099A000781DFBF70FFC002851D1F81F027A694699
:1099B0000A70407A4870B97A2980C820FBF798FB72
:1099C0003080387BA08438462E4D2838C08E2880C1
:1099D000394621482839098F41842B48FDF704FB7B
:1099E0002085608C2949FF30C33080B26084884272
:1099F0000CD949424018608428882449401C80B210
:109A00000B312880884201D30020288028887D21BE
:109A1000C9004843618C4018606500F0A3F86846AF
:109A20000088E0841249B87CC73160714200084662
:109A30000D466930FBF7A2FB6079294642001448C5
:109A4000FBF79CFBA08CFF2801D003202070F8BD01
:109A5000FFE700F04DFF0000700000204C010020E7
:109A60005A01002000040050400100204101002064
:109A70005C120020E80D00201800002000D02724F0
:109A8000600100206C01002004160020E7030000A4
:109A9000A413002070B586B014216846FBF787FB3D
:109AA00001250F4EED03002229463046FDF77FF8D1
:109AB00001200024019002946946009503943046E9
:109AC000FCF7ACFF032001900294694600950394D3
:109AD0003046FCF7A3FF022001F0EAF806B070BDA3
:109AE000000400500088704770470000F8B5044635
:109AF00000206A461080194D55222A70AA226A70E9
:109B00000322AA70661DEE702A716971144A490019
:109B10008918AC712246E81DFBF730FB002007E0F6
:109B200029186A468978128889186A461180401C6B
:109B3000B042F5DB611DA81CFCF754F801466846ED
:109B4000018029190078C87168464078087221465A
:109B50000931024800F0DCFBF8BD0000421500208E
:109B6000E80D0020FEB5FFF7A1FB2548FDF73CFA04
:109B7000244C86B2268560790A21081AC000FBF7BA
:109B80008BFD07460191A06EFBF79AFD1E4A1F4B05
:109B9000FBF7E2FC00900D463046FBF791FD2B46AB
:109BA000009AFBF7BFFB3A46019BFBF7BBFBFBF7B9
:109BB000CDFD85B2A586E08BFBF782FD124A134BE3
:109BC000FBF7CAFC06460F462846FBF779FD3246EE
:109BD0003B46FBF7A7FBFBF7B9FD81B20120C003B1
:109BE000E186814201D3091AE186854201D3281A10
:109BF000A0860349A08E096848612087FEBD000049
:109C00000416002070000020F853E3A59B843E401A
:109C1000034A1168382389B29943014311607047A0
:109C20000030014010B5FCF7CFFF10BD10B59AB061
:109C300034216846FBF7BBFA14210DA8FBF7B7FAED
:109C40001C2112A8FBF7B3FA1B4801680324E402A5
:109C5000A143C21489180160FDF744FA174801694D
:109C6000A143016106200090FF20013002900120F5
:109C70000390102004900220099040040B900001F2
:109C800000240C900A946846FDF75AFC0F200D90B2
:109C900003200E900F941094012111940DA8FDF74C
:109CA00025FB81201290032080041890149412A8A0
:109CB000FDF76AFA1AB010BD007000404010024073
:109CC00010480168821511430160C1680E4A1140B5
:109CD000C16001680D4A114001608168490849006E
:109CE000816001680122920491430160C168FD22F4
:109CF00012049143C1600021016106490448886053
:109D000070470000001002400C40FF88F6FFF6FE8E
:109D10000050000800ED00E070B5026801239B07C9
:109D2000114C124D984203D0A04201D0A84203D159
:109D30007026B2434E683243984203D0A04201D00D
:109D4000A84204D103231B029A43CB681A43802301
:109D50009A430B691A4302608A68C2620968816289
:109D60000121416170BD0000000801400014014064
:109D700010B5CB06DB0E0121046A99408C430462C6
:109D8000016A9A401143016210BD30B58468FF2515
:109D90002D021B021343AC430B432343836030BDAE
:109DA000826870239A430A4307210A4382607047FE
:109DB00030B5026A520852000262026A456883693D
:109DC0007024A3439C080B68A40023430224A243ED
:109DD0008C6845601443836149684163046230BD07
:109DE00030B5026A10239A430262036A45688269A9
:109DF00073242402A2430C682402144320229343B8
:109E00008A68456012011A4384614968816302626D
:109E100030BD30B5026AFF2301339A430262026A01
:109E20004568C3697024A3439C080B68A4002343BE
:109E300001246402A2438C68456024021443C36178
:109E40004968C163046230BD30B5026A01231B0357
:109E50009A430262036A4568C26973242402A243DA
:109E60000C68240214430122520393438A6845601C
:109E700012031A43C46149680164026230BD30B5FF
:109E8000036A046A6408640004628469F025AC43D0
:109E9000120122430A24A3430B438261036230BDB3
:109EA00030B5036A1024A34303628469036A0F2553
:109EB0002D031203AC432243A024A34309011943F9
:109EC0008261016230BD0000F8B5102405252D0720
:109ED000AC62AF20800000F0F2FEAC6101F0CEFB7E
:109EE0002F4C304F304E60670EE001F0C7FB6067CB
:109EF000FEF71CFB606C411C6164142804D92BA084
:109F000000F078FC2D48C760606FB042EDD10026AC
:109F1000666420780127FF03030000F0A4FC050419
:109F20000C192D303200012239462846FCF73FFE3D
:109F3000FFF7A6FC06E0012239462846FCF737FE6B
:109F4000FFF792FA002239462846FCF730FE18E067
:109F5000607B0122401C607339462846FCF727FECF
:109F6000FBF7FEFF002239462846FCF720FE607B07
:109F7000052806D9267004E0FEF792FE01E0FFF7FF
:109F800073FA02210E48FCF705FE002805D00020D8
:109F90000C49087001F058FAF8BD0120F8E70000FC
:109FA000700000200400FA053001CADE4457204941
:109FB00044204552524F522E0D0A000000ED00E0A1
:109FC000000400507001002010B5818CC90707D033
:109FD00001684A6801235B049A43836A1A434A6012
:109FE000818C890707D501684A6801231B049A43BD
:109FF000C36A1A434A60818C490707D501684A68D9
:10A0000001239B049A43036B1A434A60818C09071E
:10A0100007D501684A680123DB039A43436B1A435F
:10A020004A60818CC90607D50268916801231B0329
:10A030009943836B19439160818C890607D5016828
:10A040008A6801235B039A43C36B1A438A60818C3D
:10A05000490612D503685A6801210905046C8A4330
:10A0600022435A60026C8A4207D102685168032376
:10A070005B059943436C19435160818C090607D5F0
:10A0800001684A680123DB04806C9A4302434A60FA
:10A0900010BD0000F8B50446002680300660FCF7CD
:10A0A0008DFD054620680068124F000709D5012183
:10A0B0002B46002249052046009700F0A1FA00280F
:10A0C0000DD12068006840070BD501212B460022E6
:10A0D00089052046009700F093FA002801D003205C
:10A0E000F8BD2020A067E067266660342675002052
:10A0F000F8BD0000FFFFFF01F8B5154CC826E07859
:10A10000002823D16079002820D101206071114DF1
:10A11000686B0027002818D0686BC821081A0FE068
:10A120000D48E168405C61698847E068401CE06078
:10A13000E068C82800DBE760696BC820401A761E1B
:10A14000E168814201D0002EEADC6771F8BD0000B1
:10A150005400002000000240200D002070B5224C69
:10A16000E07800283FD1207900283CD101202071DF
:10A170001E4EF16900250906002933DA215662577F
:10A1800091420AD1F06940062CD5A079002829D047
:10A19000A5712089401C208124E0A179002903D1E8
:10A1A000A0710A2000F08BFD00202056CC214843EE
:10A1B0000F494218206912181279B262401C00221D
:10A1C0002061A256CC235A43895881420ADC25617A
:10A1D0002078401C207020780E2800D12570A078AF
:10A1E000401CA070257170BD540000200038014053
:10A1F000F801002010B5806A0022014640314A83F0
:10A200004A82FDF71FFE10BD70B5846AA06FE56F2E
:10A210002168896800260906002906DA212804D168
:10A2200052200653204600F06BF8206880684006F4
:10A2300006D5222D04D15A200653204600F047F8B7
:10A240002046803001681022114301602046FDF74E
:10A25000F9FD70BD10B501460968806A0968890674
:10A260001CD400225A210A5201680A68FF230133D4
:10A270009A430A6001688A68520852008A6001683D
:10A280008A6840239A438A602021C167016E0129B0
:10A2900004D101680A6810239A430A60016E0129FB
:10A2A00002D0FDF7B1FF10BD5821095AFDF7C8FDD6
:10A2B00010BD10B5806A016E012902D0FDF7A5FF1F
:10A2C00010BD5821095A4908FDF7BAFD10BD0168B3
:10A2D0000A68FF2321339A430A6001688A6852089A
:10A2E00052008A60016E012904D101680A681023B6
:10A2F0009A430A602021C1670021016641667047C8
:10A3000001680A68C0239A430A6020218167704768
:10A3100070B5164CE278002A0CD12279002A09D1B6
:10A320000122E2700025C82903DC0222A256002A7D
:10A3300001DCE57070BD0123E356CC2253430C4A87
:10A34000D1500123E356CC2673439B180A4601469D
:10A35000181DFAF713FF6078401C607060780E28B3
:10A3600000D16570A078401EA070E2E75400002084
:10A37000F8010020F8B50446016880682369E669A1
:10A3800018436369002533431843724A0B68724EC1
:10A39000334003430B602168486803231B03984341
:10A3A000E368184348602168A069914201D0236A9C
:10A3B00018438B680B263602B34303438B6067490F
:10A3C000236867488B420CD1C0688007800F06D095
:10A3D000012839D0022835D0032821D11EE00127D9
:10A3E0001FE060498B420AD1C0680C21084027D089
:10A3F000042829D0082825D00C2811D10EE093423A
:10A400000ED1C16803208002014019D001208002D2
:10A41000091A19D0091A15D0814201D1082700E084
:10A4200010274F49504840398600934232D1002FBF
:10A430000CD0022F0DD0042F10D0082F7FD126E092
:10A440000027EEE70227ECE70427EAE7FDF71CF810
:10A4500006E00968C90605D4304603E0FDF734F884
:10A46000002872D0626851005118814267D81103E8
:10A47000814264D3010E060250080023301859416E
:10A48000FAF74CFE03210902411A384A55E001202F
:10A49000C003E7E70122E369D20393422BD13B00DB
:10A4A00000F0E1F90906090C4D114D4D4D274D0005
:10A4B000FCF7EAFF09E0FCF7F7FF06E00968C906C8
:10A4C00005D4304603E0FCF7FFFF00283DD061686B
:10A4D00040004A088018FAF70BFE80B20146244A71
:10A4E000103991422BD8511C01400007400F0843FE
:10A4F00029E01046EBE73B0000F0B5F90906090C2E
:10A500002112212121232100FCF7BEFF0AE0FCF7E4
:10A51000CBFF07E00968C90606D4304604E00EE028
:10A52000FCF7D2FF002810D061684A081018FAF72B
:10A53000DFFD80B201460E4A1039914203D9012550
:10A5400003E01046F0E72168C86000206066A0665E
:10A550002846F8BD00480040F369FFEF003801408D
:10A56000401002400044004000093D00FFFC0F0085
:10A57000EFFF0000F8B5044641654030002627464D
:10A58000028380373E602220E0672546206F6035D9
:10A5900000281CD01749C162216F17480863216F3A
:10A5A00016484863206F8663236F606D9C46134690
:10A5B0002168024660462431FCF758F9002806D08D
:10A5C000102038602E752020A0670120F8BD2E7560
:10A5D00020680168FF220132114301602068816810
:10A5E000012211438160206881684022114381600B
:10A5F0000020F8BD55A20008B3A2000809A2000877
:10A60000FFB581B005460F46044660350A9E39E025
:10A61000701C37D0FCF7D2FA0499401AB04222D805
:10A62000002E20D02068016849072BD5C069C0439F
:10A63000000527D401202168C00208622068016853
:10A64000FF22A132914301602068816849084900D6
:10A6500081602020A067E06780342060002028759A
:10A66000032005B0F0BD20680168FF22A1329143AC
:10A670000160206881684908490081602020A06746
:10A68000E067EBE72068C1693846884305D00021C0
:10A6900003988142BCD00020E3E70121F8E70000E5
:10A6A00010B504491020096808620248FDF7CCFB88
:10A6B00010BD0000CC16002001490D2088707047A5
:10A6C0005400002010B5FEF7A9F9FEF7C1FAC82220
:10A6D00002490348FDF768FD10BD0000200D002071
:10A6E000CC160020F8B53E4C002321783D4A1D468B
:10A6F000082910D0072947D0062950D0052952D063
:10A70000042953D0032954D0002956D0012958D008
:10A7100002295AD05BE0A17800264A1F04E0314F9D
:10A72000BF5DFB189BB2761C9642F8DB66792779F1
:10A730009A195118E3786278C9188918C91940180C
:10A74000C0430006000E1AD1012E14D0022E16D1DD
:10A7500025482449C018FAF711FD01F08BFF642049
:10A7600000F0A6FABFF34F8F21492048C860BFF31D
:10A770004F8F00BFFDE759081046FFF7B7F9257066
:10A78000E570A570A571F8BDA1795054491CC8B2F7
:10A79000A071A178491F8842F5D1082001E06070BE
:10A7A00007202070F8BDE0700620FAE760710520F0
:10A7B000F7E7A070E5700420F3E7552807D10120E2
:10A7C000EFE7AA2803D10220EBE7032803D0257086
:10A7D000E570A570F8BD032020702071F8BD000061
:10A7E00034010020DE140020E80D00200400FA05EA
:10A7F00000ED00E010B5024A024900F0E5F910BD95
:10A80000B1B90008880100202021020C01D01021DC
:10A810001046020A01D010460839020901D010463C
:10A82000091F820801D01046891E420801D0881EE7
:10A830007047081A7047F8B5040C8BB2264682B2EE
:10A840005E430D0C1046370C584336048019002126
:10A85000794116466E43370C3604801979412646F5
:10A860006E438919F8BD30B47446641E2578641CA3
:10A87000AB4200D21D46635D5B00E31830BC184755
:10A880004900CA020243100000D004204A0D01D042
:10A8900001221043044A490D914201D1022108438B
:10A8A000012800D105207047FF0700008307FF2221
:10A8B000DB0E9A408907090E9940002808DB8308BF
:10A8C00009489B001B18186890430843186070479C
:10A8D0000007000F0838830804489B001B18D8693C
:10A8E00090430843D861704700E400E000ED00E0C9
:10A8F000BFF34F8F04490348C860BFF34F8F00BFB9
:10A90000FDE700000400FA0500ED00E0F8B504469C
:10A910004F1EC8000838211815461E4608684968A9
:10A920003A4606239A4310D02A463346FAF7ACFD3E
:10A930003A46D200083AA3181A687F1E5B68FAF7F5
:10A94000F1FC06223B469343EED1022F23D0042F85
:10A9500011D0062F2FD12A463346FAF795FDE36A28
:10A96000A26AFAF7DFFC2A463346FAF78DFD636ADE
:10A97000226AFAF7D7FC2A463346FAF785FDE369DF
:10A98000A269FAF7CFFC2A463346FAF77DFD6369E0
:10A990002269FAF7C7FC2A463346FAF775FDE368E1
:10A9A000A268FAF7BFFC2A463346FAF76DFD6368E2
:10A9B0002268FAF7B7FCF8BD002210B5134610461E
:10A9C0000149FAF7C9FD10BD0000F03F10B5FAF7D4
:10A9D000A9FC10BD002210B5134610461146FAF727
:10A9E000BBFD10BD10B50721024A00200907FAF788
:10A9F0002BFE10BD01030000034A10B50020110713
:10AA0000FAF722FE10BD000001FDFFFF02E008C8BA
:10AA1000121F08C1002AFAD170477047002001E0D8
:10AA200001C1121F002AFBD17047000001490860D4
:10AA3000704700008C01002008B5002168460170B5
:10AA40006B46012202212C2000F052FF02216846B1
:10AA500001706B4601222C2000F04AFF08BD000067
:10AA600038B504466D20694608706B4601220749D7
:10AA70002E2000F03DFF0649002C01D0054A00E0E1
:10AA8000054A2E2000F01AFF38BD0000060800001D
:10AA900006180000070600000716000038B5044637
:10AAA0006B4602220021362000F0EEFDB321230088
:10AAB000FFF7D9FE0E0F08153A3A3A3A1C273A3AF0
:10AAC0002F34483A00216846017040784108490017
:10AAD00014E06946087880088000401C04E069465C
:10AAE000087880088000801C08701DE068460278A5
:10AAF0000A40483202704178802001436846417024
:10AB000012E0684602780A40027040784106490E19
:10AB1000F4E7694648780221084303E0694648782B
:10AB2000FD210840694648706B460122002136200D
:10AB300000F0DEFE012200AB11463620013300F0AA
:10AB4000D7FE38BD69460878CF21084069462030D5
:10AB5000CAE708B5032168464170012101706B46C0
:10AB600002220021362000F0C3FE0122D20306217A
:10AB70002D2000F0A3FE012000F09AF80120FFF73D
:10AB80008DFF08BD08B5020A69464A7008706B4619
:10AB9000022204212D2000F0ABFE0320694608703C
:10ABA0006B46012206212D2000F0A2FE00206946FE
:10ABB00008706B46012206212D2000F099FE0A2123
:10ABC0002D2000F047FD08BDF8B516460F46044697
:10ABD000002503E03946B047641C6D1C207800282E
:10ABE000F8D12846F8BD0000F8B54A002B4B520DAD
:10ABF000D6182B4A0C460546142E2BDA002E12DAF4
:10AC0000284BFAF78FFB00221346FAF7E5FD40D2F6
:10AC1000002C03DA0124E40700253AE0204628430B
:10AC200037D0214C14E0214F0B46F7403B402B43DB
:10AC300031D01C4BFAF776FB00221346FAF7CCFD15
:10AC400027D2002C03DD01200005F0400419BC438D
:10AC500000251EE0332E1EDC33460027143BFF4345
:10AC6000DF40384217D00F4BFAF706FC002213469C
:10AC7000FAF7B2FD0DD2002C0ADD142E0CD03420D0
:10AC8000811B012088404019A84200D2641C05465F
:10AC9000BD4321462846F8BD641CF9E701FCFFFFCF
:10ACA0009C7500883CE4377E0000F03FFFFF0F00FA
:10ACB0007D2110B5C900484300F001F810BD002106
:10ACC00040E000BF00BF00BF00BF00BF00BF00BF2B
:10ACD00000BF00BF00BF00BF00BF00BF00BF00BF7C
:10ACE00000BF00BF00BF00BF00BF00BF00BF00BF6C
:10ACF00000BF00BF00BF00BF00BF00BF00BF00BF5C
:10AD000000BF00BF00BF00BF00BF00BF00BF00BF4B
:10AD100000BF00BF00BF00BF00BF00BF00BF00BF3B
:10AD200000BF00BF00BF00BF00BF00BF00BF00BF2B
:10AD300000BF00BF00BF00BF00BF00BF00BF00BF1B
:10AD400000BF491C8142BCD37047FFB581B01E468D
:10AD50000F46040026D00B9903980143A06A39439B
:10AD6000826807209047002818DB0A99A06A3143BF
:10AD7000826806209047002810DB25462035A979F7
:10AD8000032F01D908200143032E01D904200143D8
:10AD9000A06A826809209047002806DA0120C04393
:10ADA00005B0F0BD0020C043FAE7384600F000F9D6
:10ADB0002060304600F0FCF860600A9868700398E4
:10ADC000A870EF702E710B9868710020E8E7000002
:10ADD000F7B50446002090B000900190002C05D0FB
:10ADE0006A46062101F080FC062803DA0020C043F1
:10ADF00013B0F0BD68464078010268460078000450
:10AE00000918684680780818FAF75AFC054668461B
:10AE10000391007901026846C07800040918684669
:10AE200040790818FAF74CFC032206460F469207B1
:10AE30005C4BFAF7D1FC07D200225B4B3046394617
:10AE4000FAF714FB06460F4603229207554B284695
:10AE50000399FAF7C1FC07D20022534B2846039905
:10AE6000FAF704FB054603912068FAF729FC02462D
:10AE70000B4630463946FAF76FFB07460A20079122
:10AE8000205EFAF709FC3A46079BFAF7FDFA0646F8
:10AE900008200991205EFAF7EDFB0021C943FAF77B
:10AEA00035FAFAF771FC3246099BFAF73BFA06913C
:10AEB00008906068FAF704FC02460B46284603999E
:10AEC000FAF74AFB05461A200E46205EFAF7E4FB25
:10AED0002A463346FAF7D8FA0C9009911620205EDC
:10AEE000FAF7DAFB099B0C9AFAF71CFA05910A901B
:10AEF0002A46334638460799FAF7C6FA059B0A9A56
:10AF0000FAF7C2FA05910A901420205EFAF7C4FB02
:10AF10003A46079BFAF7B8FA07461C200791205ECD
:10AF2000FAF7BAFB2A463346FAF7AEFA0E900B91BF
:10AF30001820205EFAF7B0FB0B9B0E9AFAF7F2F995
:10AF40002A463346FAF7A0FA0B910E902069FAF7D9
:10AF5000A3FB0B9B0E9AFAF7E5F92A463346FAF75C
:10AF600093FA05460E46E068FAF796FB2A46334602
:10AF7000FAF7D8F93A46079BFAF7D4F9059B0A9AEB
:10AF8000FAF7D0F901229207084BFAF77DFA024648
:10AF90000B46129C0898069903C411980CC0002017
:10AFA00026E70000FFFF5F4100007041E17A843F27
:10AFB00000B50121C9040300FFF755FC081A050874
:10AFC0000B0E1114171A0320C00400BD0720C00483
:10AFD00000BD0F20C00400BD1F20400300BD3F2066
:10AFE000400300BD7F20400300BDFF20400300BDA3
:10AFF000084600BDFEB5264F0D4604000FD0002DBB
:10B000000DD0264600202036B071F07129680D2041
:10B010008847002801DA7800FEBD102801D03846A4
:10B02000FEBDA562E968002901D028208847204696
:10B0300000F030F80028F3DBA06AA52182680E201A
:10B040009047A06A962182680F209047A06A02214B
:10B05000826862209047A06A002182680E20904793
:10B06000A06A002182680F209047717930200191F9
:10B0700000900623202201212046FFF766FE0028CB
:10B08000CEDB204600F0AEF80028C9DB0020FEBD74
:10B09000FFFFFFFF10B586B0044614216846FAF79B
:10B0A00086F8002C7ED0A06A122143686A461020E0
:10B0B0009847122877D16846007801220101684636
:10B0C000407812030009081843492081884201DDB5
:10B0D000801A20816846837840780007000D181890
:10B0E0006081884201DD801A608168460079012212
:10B0F00001016846C07812050003091868464079C6
:10B10000000908183549E060884201DD801AE060D6
:10B11000684640790007030B6846807900021B18D7
:10B120006846C07918182061884201DD801A2061C4
:10B130006846417A007A0002081802B228480121C4
:10B140000904A282824201DD521AA2826A46D37A9F
:10B15000927A12029A1812B2E282824201DD521AE7
:10B16000E2826A46537B127B12029A1812B2228341
:10B17000824201DD521A22836A46D37B927B1202FD
:10B180009A1812B26283824201DD521A62836A46C1
:10B19000537C127C12029A1812B2A283824204DDFE
:10B1A000501A01E00BE008E0A083A06A01682820A3
:10B1B0008847002806DA0120C04306B010BD0020F1
:10B1C000C043FAE7C011C0072034002800D0802017
:10B1D00060710020F1E70000FF070000FFFF07009B
:10B1E000FF7F000010B5040009D0A06A0721826823
:10B1F00008209047002805DA0120C04310BD002038
:10B20000C04310BD072020342070002010BD000076
:10B21000FEB504460020019000906079734940001B
:10B220000E5A61782578491E7148CFB20163042D0A
:10B2300077D0072D75D000210291217801736C49D8
:10B24000E379012292058969002B6CD091438161D9
:10B250006748217A4173217A82698907890B0A43F9
:10B2600082610021042000F034FB324661492E2027
:10B2700000F024FB3846FFF7F3FB5F4E0522705DBC
:10B28000810040185D49431807212B2000F030FB56
:10B290005B49029801220B180B21282000F028FBA3
:10B2A000705D584980000A580C21282000F011FBDD
:10B2B000E079554980004018A1794900425A02219D
:10B2C000272000F0FBFA51487E00825B04212720F2
:10B2D00000F0F4FAE079002829D0A07804282CD0D6
:10B2E00028206946087220220621272000F0E6FA6D
:10B2F00002AB01222621272000F0FAFA4449380146
:10B300004018E178890042580821272000F0E1FA2E
:10B31000A17A601C627A0902114313D016E000E0A2
:10B3200001E0012188E71143F608816190E764227A
:10B330000621272000F0C2FAE0E7102069460872D3
:10B340000246D1E733490172090A4172417A007A13
:10B350000A0202432021272000F0B0FA2E4F0C21D0
:10B3600023203A6800F0B5FAF019828804212320DE
:10B3700000F0A4FAA07900280BD0E0792749012237
:10B3800043180021212000F0B3FA0320019001208E
:10B3900000902A07120F10010243607800218007F5
:10B3A000000B024301980005024300984004024349
:10B3B0002079C006400902436079C00602431F207D
:10B3C00000F087FAA0786178012308430204084856
:10B3D000DB030261E179490319430A430261002159
:10B3E000082000F076FA0020FEBD00001CC800080E
:10B3F000BC01002004280000C4C70008240000206D
:10B4000042000020CCC70008ECC70008F8C70008BD
:10B41000FCC7000841100000E4C7000844000020F9
:10B4200038B50C4607498A8B002102432C2000F0D6
:10B4300045FA684604706B46012206212C2000F074
:10B4400057FA38BDBC01002010B5FFF7F5FA10BD62
:10B4500010B504460421362000F0FCF80121C90291
:10B46000002C01D0084300E0884302460421362026
:10B4700000F02FFA10BD000038B540206946087072
:10B4800000210E2000F0E6F80446002211460E20AE
:10B4900000F01FFA6B46012200210D2000F028FA6F
:10B4A000074A00210F2000F014FA00F0EDF92246BF
:10B4B00000210E2000F00DFA02480021017338BD72
:10B4C000F8FF2724DC010020FEB50546042069466C
:10B4D0000870514C0020607521462031206348716E
:10B4E0000873A0836063A06300F0C8F84B4E20602F
:10B4F00002E000F0C3F82060B042FAD10020FFF76C
:10B50000CDFA00F0BBF8464E20603078242801D9EF
:10B51000243806E00621F9F7EBFD0622101A400157
:10B520000843020601040A4301020A430243B260CF
:10B53000706000211E2000F0CCF900F09FF8206020
:10B540006B4601220021242000F0D2F91E20FFF7D3
:10B5500019FB86B2300AA0730420FFF713FB0746DD
:10B5600000F08CF820603806000E0DD002206946ED
:10B57000087101AB012212212D2000F0B9F9A08B36
:10B58000012109030843A08300F078F82060062019
:10B59000FFF7F8FA60600720FFF7F4FAA060F00602
:10B5A000C00E207501D110202075C0B200F0DCF96A
:10B5B000E80707D0FFF7CDFAA08B0121C9020843A5
:10B5C000A0830AE00521362000F02EF81549084036
:10B5D00002460521362000F071F90120FFF75EFADE
:10B5E0000021042000F036F8A0610021262000F0A0
:10B5F00031F815218903084302460021262000F076
:10B6000068F900222621362000F058F900F036F8BB
:10B6100020600020FEBD0000BC0100203001CADE19
:10B6200018000020FFFD000038B5094C89B280B237
:10B630006B46022200F028F8002806D168464078C0
:10B64000010268460078081884B2204638BD000020
:10B65000FFFF000038B50024E44389B280B26B4696
:10B66000042200F011F8002806D103216846435C4B
:10B670002202D418491EFAD5204638BD10B5002143
:10B680000846FFF7E7FF10BD38B5002909D0402470
:10B6900020436C462070C8B27F2906D86070022013
:10B6A0000AE069460870012006E0802420436C46C9
:10B6B0006070C809A0700320694600F0B5FF38BD6E
:10B6C00010B5144603460A4621461120FFF7DCFF59
:10B6D00010BD10B50346052200211520FFF7D4FF49
:10B6E00010BD10B50346052200211720FFF7CCFF3F
:10B6F00010BD38B5054600206946087000F0C4F852
:10B70000FF2401342246002D01D003221202002121
:10B710000D2000F0D3F8002D13D06B460122032139
:10B720000F20FFF7B1FF68460078000709D5FFF743
:10B73000A3FE224600210D2000F0C0F80020C043E7
:10B7400038BD002038BD10B5024601210A2000F0A6
:10B75000C0F810BD10B5044600211A20FFF77AFF8B
:10B76000000D22030005120B024300211A2000F0F5
:10B77000B0F810BD10B5024602492E2000F09EF828
:10B7800010BD000004180000F8B505466B46012204
:10B7900003210420FFF778FF0126114C3607002D06
:10B7A0000DD02A4600210C2000F088F86946087860
:10B7B0001021084369460870A069304307E06946D4
:10B7C0000878EF21084069460870A069B0430B462D
:10B7D000A06101220321042000F08AF8F8BD0000D6
:10B7E000BC01002010B502460021182000F066F8C8
:10B7F00010BD0000F8B50746002568460570B8077B
:10B80000204C2E4600280ADA8020694608706B46D4
:10B81000012200210D2000F06BF801202073F807B1
:10B820006946087821D006210843694608706B46AE
:10B83000012200210D2000F05BF803210F20FFF70B
:10B84000F3FE8121C900084219D0402069460870E2
:10B850006B46012200210D2000F04AF80020FFF77E
:10B86000F7FD00252673ED4309E0022108436946F0
:10B8700008706B46012200210D2000F039F828469F
:10B88000F8BD0000DC0100201CB56B46012203213D
:10B890000F20FFF7F9FE684600784022C1091040EA
:10B8A000C9014000814208D0012069460871024662
:10B8B00001AB03210D2000F01BF81CBD08B56B4641
:10B8C0001A70120A5A7089B280B2022200F010F87F
:10B8D00008BD38B500236C46E254120A5B1C042BE9
:10B8E000FADB89B280B22346042200F001F838BDA9
:10B8F00038B58024002909D0C02528436D4628701A
:10B90000C8B27F2907D86870022009E02043694641
:10B910000870012004E020436870C809A870032063
:10B92000694600F02BFF38BD10B5144601231218EC
:10B930009B029A4202D90020C04310BD0B46821ED2
:10B9400021460920FFF7D4FF002010BD10B5054A9D
:10B950008905126901430A4300210820FFF7B9FF56
:10B96000002010BDBC01002038B504466B46012202
:10B970000E212B20FFF788FE68460078E10640097B
:10B980004001C90E0143684601706B4601220E2139
:10B990002B20FFF7ADFF38BD10B5002142541C0627
:10B9A000120A22431B0A491C0429F7DB10BD0000C0
:10B9B00013B501231A4669460248FCF727FC009894
:10B9C0001CBD0000CC1600207CB50024254668462E
:10B9D000FFF77FFE04206946220E2D021543220246
:10B9E0000C5C1443401EF7D5204629467CBD7CB52F
:10B9F000002425466846FFF774FE04206946220E9F
:10BA00002D02154322020C5C1443401EF7D520463C
:10BA100029467CBDFBF7E0F8FEF708F9FDF712F8C0
:10BA20003F494048002522C005608561C5613E4907
:10BA30000562C1600838FBF761FAFCF7EFFFFDF71C
:10BA400007F9FDF7A3F8FCF7B5FF05240122240749
:10BA5000D1032046FBF7ABF8FDF798FEFCF792FE0A
:10BA6000FAF79CF8FAF71EF9FAF7ECF8FCF750FC35
:10BA70000721A015FFF7D4FCFFF7E6FC0122110314
:10BA80002046FBF794F82748C8222849C830FCF71D
:10BA90008BFBFCF725FE264F264E274C38780028D6
:10BAA0000FD13078002801D003280AD10121C90222
:10BAB0002248FBF76FF8002803D101210846FBF765
:10BAC00031FBE078002828D06078002825D0E57088
:10BAD00072B620780F280AD901201849000388611E
:10BAE000FEF7F2F901201549000388620CE00122FB
:10BAF00051031248FBF75BF8FEF7E6F9012100223B
:10BB000049030E48FBF753F862B6FCF70FFD208C93
:10BB10000028C3D0401E2084C0E7FCF707FDBDE726
:10BB2000007C004004160020FFFF0000200D0020D4
:10BB30005A000020840000203C0100200004005036
:10BB400010B586B01848FBF75CF914216846F9F780
:10BB50002EFB164800900320019000200290052043
:10BB600069460007FAF75AFF69461148FAF756FF87
:10BB700069461048FAF752FFFCF7B2FD012108466A
:10BB8000FBF7D0FAFF2401342046FBF7A3FA0A4959
:10BB900008680422104308602046FBF7ABFAFBF765
:10BBA000B1FA06B010BD000004160020FFFF00002F
:10BBB00000040050000800500070004010B5012241
:10BBC000920217491748FAF7F1F815481649028802
:10BBD0008A4223D0018004218180FF21F531C18078
:10BBE0000A21018100211E224181D243828101224A
:10BBF000C28181834323C38602230387782343873B
:10BC00008287C28702464032118451849184C18365
:10BC1000918014238382118200F02CFD10BD00005E
:10BC2000E80D002000FC0008AA550000F0B51FB484
:10BC300096B084460C460246199D18980390490018
:10BC400068006300490840080193002A01D00126DA
:10BC500000E000269E19FE4BF6185B109E422BD387
:10BC60006E00039F0296002F00D00127F719F84EAF
:10BC7000F84BBE199E421FD3039E0346F64F334333
:10BC800009D03B469C4201D1002A04D0019B002AE6
:10BC900005D0012604E0002039461BB0F0BD002687
:10BCA0009E19EE4B9E4207D8039F029E002F00D0A4
:10BCB0000127F6199E4207D92B4660462146189A5D
:10BCC000FEF784FE1BB0F0BD0023002C29DAE44E01
:10BCD000B04226DAE34EB04201DB022321E0DE4E21
:10BCE000B0421EDBE04E070DBE19142E09DD3427CD
:10BCF000BF1B039EFE400196BE40039FBE420BD079
:10BD00000FE0039F002F0CD11427BF1B0646FE40F7
:10BD10000196BE40864204D1019BDE07F60F022346
:10BD20009B1B0E46164318D1002D16DA002C03D0AB
:10BD3000022B01D0012B06D00220FEF777FEFEF782
:10BD40003BFE1BB0F0BD0220FEF770FEFEF734FE96
:10BD50000122D20751401BB0F0BD039E002E61D1DD
:10BD6000BF4EB04220D1C148844201D1002A08D040
:10BD7000B948814209DB002D10DB189829461BB019
:10BD8000F0BD0020B4491BB0F0BD002D06DA012241
:10BD90002946D207189851401BB0F0BDB4497944E8
:10BDA000086849681BB0F0BDAB4FB84225D1002DE3
:10BDB0001FDA002904D0B14212D1002A09D018E0BC
:10BDC000002A72D1A649E20F0020D20711431BB00E
:10BDD000F0BD0020E20F0146D20711431BB0F0BDB9
:10BDE000B14206DA234600203946F9F7B5FB1BB00D
:10BDF000F0BD104621461BB0F0BDB14212DA01265B
:10BE0000B607B54203D1234610461946FEE3994EC4
:10BE1000B54207D1261E05DB1046314600F040FC36
:10BE20001BB0F0BD67007F081646002A40D10029EC
:10BE30000AD08B4A914229D1002C0EDD002D1CDB4B
:10BE4000002011461BB0F0BD022B16D0002C14D0E0
:10BE5000012B12D1002C14DB0FE0002C28DA002D6E
:10BE600009DB012B03D000207D491BB0F0BD002071
:10BE700081491BB0F0BD012B03D0002001461BB04F
:10BE8000F0BD00200121C9071BB0F0BD724A9142EC
:10BE90000ED1002C01DA002B17D0022B06D0002087
:10BEA000C043F9F7F9FB1BB0F0BD90E20120F8E7C1
:10BEB000E217521C94461A4307D000220892664C9F
:10BEC00062465B1E1A4307D009E00120FEF7AEFD73
:10BED000FEF780FD1BB0F0BD0022644C0892674A5B
:10BEE00090427DDD664B674A98421FDD914202DC3D
:10BEF000002D05DB4DE05848814217DB002D48DD61
:10BF00000220FEF793FDFEF76DFD05460E4600226A
:10BF1000534B21460898F9F7B7FA084671004908CB
:10BF2000C00FC007014328461BB0F0BD914215DA8F
:10BF3000002D2EDA0220FEF779FDFEF753FD0546AF
:10BF40000E460022464B21460898F9F79DFA7200EA
:10BF50005208C80FC0070243114617E03E4B9942F2
:10BF600023DD002D15DD0220FEF760FDFEF73AFD12
:10BF700005460E4600223A4B21460898F9F784FA06
:10BF8000084671004908C00FC007014328461BB08E
:10BF9000F0BD0220FEF74AFDFEF72EFD49004908DC
:10BFA000E20FD20711431BB0F0BD002230463946E4
:10BFB000F9F75CFA012205460E46D243F9F744FB35
:10BFC000314A324BF9F758FA2A463346F9F75CFA08
:10BFD0000022284BF9F750FA07462A46334600E07C
:10BFE00064E0039110461946F9F74EFA3A46039B6E
:10BFF000F9F74AFA0746032209915207244B2846CB
:10C000003146F9F741FA07910C90224A204B384605
:10C010000999F9F739FA074601911F4A1F4B28463B
:10C020003146F9F731FA3A46019BF9F71FFA07460C
:10C030000B460246099107990C98F9F773F9002508
:10C040000E462846079B0C9AF9F710FA3A4627E065
:10C05000FFFF1F00FFFF0F000000F03F0000E0FFA8
:10C060000000F07F0000404301FCFFFF0000F0BF34
:10C07000560B00000000E03F0000F0FF0000E04130
:10C080000000F043FFFFEF3F555555555555D53F3F
:10C090004715F73FFE822B6544DF5DF80BAE543E3B
:10C0A000099BF9F7E9F902460B4652E10125002008
:10C0B0002D05A94207DA352230463946F9F7C4FA88
:10C0C00006463420C0430A151218FE481018039083
:10C0D0000803FD49000B01430F46FC49884201DC7F
:10C0E000002003E0FA49884202DA0120119005E0BD
:10C0F000002011900398401C7F1B03901198059716
:10C10000C200F4480F9278448018436802683946A8
:10C1100030460D930292F9F7A9F907910C90304639
:10C120000D9B029A0599F9F7FDF802460B4600208F
:10C13000E549F9F711FA09910490079B0C9AF9F770
:10C14000A3F9129000201090E3480D46784400684F
:10C150000E90012178104907084311990D9B89041D
:10C1600040180121C90447183946029A0E98F9F778
:10C170007DF93246059BF9F77FF902460B462946C1
:10C180001098F9F781F9064602913B4629460E9A26
:10C190001098F9F779F9079B0C9AF9F76DF932467F
:10C1A000029BF9F763F9099B049AF9F76DF9059178
:10C1B000129A0A902B4610461946F9F765F9064679
:10C1C0000246C6480F460B4606217844FEF79EFB02
:10C1D00032463B460091049010461946F9F754F94F
:10C1E000009B049AF9F750F906460F462B4619466C
:10C1F000129A1098F9F796F8059B0A9AF9F744F9FC
:10C2000032463B46F9F78EF8109A079104902B4678
:10C2100010461946F9F738F9B14E00223346099114
:10C220000290F9F77FF8079B049AF9F77BF8002052
:10C230000746024633460091F9F718F9099B029A1E
:10C24000F9F714F9079B049AF9F716F906460D91C8
:10C250003A462946009B1098F9F716F907910C9079
:10C260002B463046129A0D99F9F70EF905460E46FF
:10C270003A46009B05990A98F9F706F933462A468B
:10C28000F9F750F802460B460746099107990C98B2
:10C29000F9F748F800250E462846079B0C9AF9F74F
:10C2A000E5F83A46099BF9F7E7F8074607220991AE
:10C2B00052078C4B31462846F9F7E6F80791009073
:10C2C000894A884B38460999F9F7DEF80746019103
:10C2D000864A874B31462846F9F7D6F83A46019BFD
:10C2E000F9F720F8834B7B440F9A9B181A685B6818
:10C2F000F9F718F8029009910398F9F7CDF905912B
:10C300000490099B029A07990098F9F70BF87A4B69
:10C310007B440F9A9B181A685B6817460393F9F7DA
:10C3200001F8059B049AF8F7FDFF0E462846059B89
:10C33000049AF9F79BF83A46039BF9F797F8079B9D
:10C34000009AF9F793F8099B029AF9F795F80246D3
:10C350000B46199900200C900F461898F9F794F89D
:10C36000029104903B460C9A19991898F9F77EF8B7
:10C370002A463346F9F788F8029B049AF8F7D2FF69
:10C3800009910E902A46334639460C98F9F77CF805
:10C3900006460F46099B0E9AF8F7C4FF574A0D460A
:10C3A000914220DB5242AA18024310D132463B464A
:10C3B000F9F75CF804900391514A524B09990E9891
:10C3C000F8F7B0FF039B049AF9F706FA1ED2022091
:10C3D000FEF72CFBFEF706FB49004908E20FD207E7
:10C3E00011431BB0F0BD6A00474B52089A420DD36F
:10C3F000464AAA18024300D0CBE532463B46F9F73D
:10C4000035F8099B0E9AF9F7E7F9F5D9680000238A
:10C4100040082C490393020D3D4B5218984223DDEE
:10C4200001200005521CD04042195000400D401818
:10C4300038497944096813468C463749C1408B43D3
:10C4400012030121120B090551181422101AC140C0
:10C450000391002D01DA4842039062463046394686
:10C46000F9F704F806460F4632463B4609990E98FE
:10C47000F8F758FF00252A46284B28460591F9F77A
:10C4800003F807910C90264A264B28460599F8F7A1
:10C49000FBFF0091029032463B4628460599F8F78B
:10C4A000E5FF099B0E9AF8F7E7FF1F4A1F4BF8F7C5
:10C4B000EBFF009B029AF8F735FF07460B46024652
:10C4C000099135E001FCFFFF0000F03F8E9803006A
:10C4D0007AB60B0066070000A8070000D20600002D
:10C4E0000000084009C7EE3FFD033ADCF5015B148C
:10C4F000E02F3EBEA60500006C0500000000904045
:10C50000FE822B654715973C00CC904000346F3F6E
:10C510000000E03FC2040000FFFF0F00432EE63F93
:10C52000396CA80C615C20BEEF39FAFE422EE63F62
:10C5300007990C98F8F7F6FE05460E46079B0C9AED
:10C54000F8F794FF3A46099BF8F796FF09912A46B7
:10C5500033460E9010461946F8F796FF07460246F6
:10C560002F480B46059105217844FEF7CFF93A464E
:10C57000059BF8F789FF2A463346F8F77DFF074603
:10C58000019128463146099B0E9AF8F77DFF099BD9
:10C590000E9AF8F7C7FE012304910C9000229B0726
:10C5A00038460199F8F762FF05910E903A46284601
:10C5B0003146019BF8F768FF059B0E9AF8F7CCFF10
:10C5C000049B0C9AF8F752FF2A463346F8F74EFFC1
:10C5D0000022144BF8F750FF064603980D4600055D
:10C5E00041190915002912DC30462946039AF9F74A
:10C5F0002BF8FEF745F9042801D1FEF7FDF9304686
:10C600002946039AF9F720F8064601E004E02918C4
:10C610000B46324621460898F8F736FF1BB0F0BDAE
:10C62000640300000000F03FF0B58C4600251026A2
:10C63000052109078E620E4C08E067467F5DE760C2
:10C64000A768FF07FCD0E7681F706D1C8542F4DB0C
:10C650000020074606E0E760A568ED07FCD0E56826
:10C660001D54401C9042F6D38E610020F0BD0000A6
:10C670000030014070B572B60124074DA402214676
:10C680002846F9F779FB002804D0224603492846BA
:10C69000F9F716FC62B670BD00FC0008E80D00203A
:10C6A000F8B506460C46F9F7A5F9051E0F4600D069
:10C6B0000120014349000B484908411AC90F0DD018
:10C6C000002E01D0012100E000210C436100490847
:10C6D000401AC00F02D10120FEF7A8F928463946BA
:10C6E000F8BD00000000F07FF8B515460E4607467D
:10C6F000002407E03819C0B200F008F8641C287064
:10C70000E4B26D1CB442F5D33046F8BD10B5044612
:10C71000FBF7A8FEEE20FBF778FEFBF7DCFE2046D9
:10C72000FBF773FEFBF7D7FEFBF79CFEEF20FBF752
:10C730006CFEFBF7D0FE0020FBF73AFE0446FBF749
:10C74000ACFE204610BD704770B50D460446FBF7A1
:10C7500089FEEE20FBF759FEFBF7BDFE2046FBF7F6
:10C7600054FEFBF7B8FE2846FBF74FFEFBF7B3FE7F
:10C77000FBF793FE0A20FEF7A2FA70BDF0B5002584
:10C78000102605279C463F070B46BE620C4C06E070
:10C79000595DE160A168C907FCD0E1686D1C854264
:10C7A000F6DB002007E06146095CE160A168C9078B
:10C7B000FCD0E168401C9042F5D3BE610020F0BD82
:10C7C000003001400000010203040005405C00004D
:10C7D000A05C0400C06C0800805C0400E03F1E0008
:10C7E000E07D1E0007A9022570889B880A001600BC
:10C7F000010006000100020087008D002D001A31A3
:10C8000052001A339A001A351D011A376B003B315A
:10C81000BE003B335E013B3596023B370000995921
:10C820009959EB518F421E45142E0080EB51F5288B
:10C830003333E13A703DE13AC235852BC2353333AB
:10C84000C235C235AE47E13A5138A3305138000005
:10C8500000000000000001020304060708090304A9
:10C8600006080C101820300000000001020304002C
:10C87000000000000000F03F000000000000F83F52
:10C8800000000000000000000000004003B8E23F8C
:10C89000000000000000000006D0CF43EBFD4C3E3E
:10C8A000033333333333E33FFFAB6FDBB66DDB3F33
:10C8B0004D268F515555D53F01411DA96074D13F7B
:10C8C00065DBC9934A86CD3FEF4E454A287ECA3F75
:10C8D0003E5555555555C53F93BDBE166CC166BFF7
:10C8E0002CDE25AF6A56113FF16BD2C541BDBBBEF0
:10C8F000D0A4BE726937663E000000000000000050
:10C9000020C900080000002090010000BC5A000867
:10C9100084C9000890010020681A00001CAA0008C1
:10C920000124130704380D091E08054008260910C4
:10C930004008560A131D043B08BE0516D8BC40101B
:10C94000085201033AC842077052030CE5800C1BE1
:10C950000202DD140901022281F01F668104988918
:10C960009686967982159803981498879674977886
:10C9700082439788967197778249F10139293F92CE
:04C9800004922000FD
:04000005080050C1DE
:00000001FF
